:100000004CC4000079C4000077C4000075C400002F
:100010000C94990F71C400000C94250C0C94710B76
:100020006BC4000069C4000067C4000065C4000020
:1000300063C4000061C400005FC400005DC4000030
:100040005BC4000059C400000C94F72155C40000A3
:1000500053C4000051C400004FC400004DC4000050
:100060004BC4000049C4000047C4000045C4000060
:1000700043C4000041C400003FC400003DC4000070
:100080003BC4000039C4000037C4000000000C006D
:100090001800240030003C004800540060006C0050
:1000A0007800840090009C00A800B400C000CB0041
:1000B000D600E100EC00F70002010D011801230158
:1000C0002E01390144014F015A01650170017A0185
:1000D00084018E019801A201AC01B601C001CA01E0
:1000E000D401DE01E801F201FC010602100219024E
:1000F00022022B0234023D0246024F0258026102E4
:100100006A0273027C0285028E029702A002A80294
:10011000B002B802C002C802D002D802E002E8026F
:10012000F002F80200030803100318030C0C0C0C77
:100130000C0C0C0C0C0C0C0C0C0C0C0C0B0B0B0B03
:100140000B0B0B0B0B0B0B0B0B0B0B0B0A0A0A0A03
:100150000A0A0A0A0A0A0A0A0A0A0A0A0909090903
:100160000909090909090909090909090808080803
:1001700008080808080808080808080896979A9BBD
:100180009D9E9FA6A7ABACADAEAFB2B3B4B5B6B7AC
:10019000B9BABBBCBDBEBFCBCDCECFD3D6D7D9DAD3
:1001A000DBDCDDDEDFE5E6E7E9EAEBECEDEEEFF2E6
:1001B000F3F4F5F6F7F9FAFBFCFDFEFF0001FFFF93
:1001C0000203FF040506FFFFFFFFFFFF0708FFFF15
:1001D000FF090A0B0C0DFFFF0E0F10111213FF1475
:1001E00015161718191AFFFFFFFFFFFFFFFFFFFF8C
:1001F000FF1BFF1C1D1EFFFFFF1FFFFF2021FF2213
:10020000232425262728FFFFFFFFFF292A2BFF2C69
:100210002D2E2F303132FFFF333435363738FF394A
:100220003A3B3C3D3E3F0000211042206330844079
:10023000A550C660E770088129914AA16BB18CC1B5
:10024000ADD1CEE1EFF13112100273325222B5522C
:100250009442F772D662399318837BB35AA3BDD305
:100260009CC3FFF3DEE36224433420040114E664FC
:10027000C774A44485546AA54BB528850995EEE555
:10028000CFF5ACC58DD55336722611163006D7760C
:10029000F6669556B4465BB77AA719973887DFF7A5
:1002A000FEE79DD7BCC7C448E5588668A7784008D4
:1002B000611802282338CCC9EDD98EE9AFF94889F5
:1002C00069990AA92BB9F55AD44AB77A966A711A6C
:1002D000500A333A122AFDDBDCCBBFFB9EEB799B45
:1002E000588B3BBB1AABA66C877CE44CC55C222CBC
:1002F000033C600C411CAEED8FFDECCDCDDD2AAD95
:100300000BBD688D499D977EB66ED55EF44E133E4B
:10031000322E511E700E9FFFBEEFDDDFFCCF1BBFE4
:100320003AAF599F788F8891A981CAB1EBA10CD1BE
:100330002DC14EF16FE18010A100C230E3200450C6
:10034000254046706760B9839893FBA3DAB33DC339
:100350001CD37FE35EF3B1029012F322D232354216
:10036000145277625672EAB5CBA5A89589856EF5C9
:100370004FE52CD50DC5E234C324A0148104667466
:10038000476424540544DBA7FAB79987B8975FE719
:100390007EF71DC73CD7D326F2369106B0165766B6
:1003A0007676154634564CD96DC90EF92FE9C899A1
:1003B000E9898AB9ABA94458654806782768C01806
:1003C000E1088238A3287DCB5CDB3FEB1EFBF98B79
:1003D000D89BBBAB9ABB754A545A376A167AF10A56
:1003E000D01AB32A923A2EFD0FED6CDD4DCDAABD89
:1003F0008BADE89DC98D267C076C645C454CA23CA6
:10040000832CE01CC10C1FEF3EFF5DCF7CDF9BAF58
:10041000BABFD98FF89F176E367E554E745E932EF5
:10042000B23ED10EF01E787C3C1E1E1E1E1E3E3EAD
:10043000FEFCFCF8F0E0800000000000000000007E
:1004400080E0FFFFFFFF7F1F00000000FFFFFFFFB6
:10045000FF07070303010100000000000078FCFC17
:10046000FCFC7800000000000000000000C020102C
:1004700008080402020201010101F00E010000005F
:10048000000000607070000000000F70800000002D
:100490000000804020101008080800000003040835
:1004A000101020404040808080800F70800000004D
:1004B0000000081020404080808020202020202044
:1004C000202020202020202020202020202020004C
:1004D0002049646C6500205265616400577269743C
:1004E0006500547261636B202020205369646500AD
:1004F000313434304B204469736B436F7079206919
:100500006D616765003830304B204469736B436F11
:10051000707920696D616765003430304B20446923
:10052000736B436F707920696D6167650031343496
:10053000304B2072617720696D616765003830301B
:100540004B2072617720696D616765003430304BF4
:100550002072617720696D61676500696D6167650B
:10056000206E6F7420636F6E746967756F757300AA
:100570006572726F72206F70656E696E6720696D4B
:1005800061676500504C454153452057414954002F
:100590003130313031303130313031302E2E2E008B
:1005A0003031303130313031303130313031300074
:1005B000202020205550444154494E472043504C60
:1005C000442020202000436F6E74726173743A20BF
:1005D0000053454C4543543A2053617665004E45DF
:1005E00058543A204461726B657200505245563A35
:1005F000204C69676874657200626567696E0052B5
:10060000656C6561736520627574746F6E732074B8
:100610006F00434F4E54524153542041444A555366
:10062000544D454E54004170702056657273696F89
:100630006E20312E302051002020202020464C4FAB
:1006400050505920454D5520202020202000534453
:100650002052454144204552524F52205200666973
:10066000726D776172652E78766600436F756C6483
:10067000206E6F74206F70656E00434845434B20B9
:1006800050494E53202D2044454641554C5400437B
:100690004845434B2050494E20434C4B4F2D48007A
:1006A000434845434B2050494E20434C4B4F2D4C23
:1006B00000434845434B2050494E20524553455432
:1006C00000434845434B2050494E20454A4543543A
:1006D00000434845434B2050494E20435552525FFA
:1006E0005349444500434845434B2050494E20520E
:1006F000445F41434B00434845434B2050494E2003
:100700005752455100434845434B2050494E2053D2
:100710005445505F52455100434845434B20504992
:100720004E20535445505F44495200434845434B83
:100730002050494E53202D20414C4C0046415441FD
:100740004C204552524F5220202020202020202093
:1007500020005752495445204552524F52202020E4
:10076000202020202020200000000000170003008F
:10077000031F0A1F0A1F050904120F171C00030399
:10078000000E11110E00050205040E0410080004ED
:1007900004040010001804031E110F021F00191595
:1007A0001215150A07041F1715091E151D19050333
:1007B0001A150B17150F000A00040C04040E1F0A6B
:1007C0000A0A1F0E040115030E15161E051E1F151D
:1007D0000A0E11111F110E1F15151F05050E151DEF
:1007E0001F041F111F1108100F1F041B1F10101FC3
:1007F000061F1F0E1F0E110E1F05020E191E1F0DC4
:1008000016121509011F010F101F0718071F0C1FD3
:100810001B041B031C031915131F101002040810DE
:10082000101F0406041010100003031A161C1F12D8
:100830000C0C12120C121F0C1A16041E050C2A1E88
:100840001F021C001D0010201D1F0C12111F101E66
:100850000E1E1E021C0C120C3E120C0C123E1C0230
:1008600002141E0A021F120E101E0E180E1E1C1E4F
:10087000120C1206281E1A1F16041B11001F00114D
:100880001B04080C047C3C3E5E2B3D3F2F5B5D3B14
:100890002C2A225C0000E221E62111241FBECFEFAA
:1008A000D0E4DEBFCDBF13E0A0E0B1E0E6EAF2E8BD
:1008B00000E00BBF02C007900D92A636B107D9F732
:1008C00018E3A6E6B3E001C01D92AB32B107E1F731
:1008D00018E000E0C8E9D8E040E006C022974109EE
:1008E000FE014BBF0E94F93DC639D1074007B1F761
:1008F0000E94791C0C94424183CB2F923F924F92DD
:100900005F926F927F928F929F92AF92BF92CF929F
:10091000DF92EF92FF920F931F93DF93CF93CDB7A8
:10092000DEB72D970FB6F894DEBF0FBECDBF8B019B
:100930004A013E010894611C711CD301E4E2F1E01C
:100940002DE001900D922150E1F7BB244424AA240C
:1009500052E8552E42E2E42EF12CE80EF91E3EE05C
:10096000C32ED12CCC0EDD1E22E8222E312C280CD9
:10097000391CC701B80140E250E00E94482980328A
:100980009105A1F4D8011B968C911B9790E09C01D6
:100990002F7330702F30310559F183FD23C0F801DA
:1009A0008081853E19F1882309F05AC0D4011C9238
:1009B00080E02D960FB6F894DEBF0FBECDBFCF916D
:1009C000DF911F910F91FF90EF90DF90CF90BF903C
:1009D000AF909F908F907F906F905F904F903F90DF
:1009E0002F900895F8018081882301F3BB24C1CFA3
:1009F000BB2021F58C91982F907E903409F0B9CFCF
:100A00009FE1A92EA8221D964C90F1011082A5E726
:100A1000B0E085E7582EF301AD01480D591D8191D5
:100A20009801280F311DD9018C91DA018D93AD0108
:100A3000EC15FD05A1F7BB24B3949BCFD8018C9195
:100A4000AA948A1599F61D968C911D97841571F6B6
:100A5000552009F48ECFB3EF5B0EA52DB0E0DBCFB0
:100A60008E3221F2BB2081F031962BE090E001C064
:100A70008191392F3795332737959695932B980F7A
:100A80002150B1F7941531F0C801B4010E948828B3
:100A900081E08FCFFA2DF130B9F7452D50E0433882
:100AA0005105B4F79A0160E080E090E0880D991D4F
:100AB000280D391DD9012C91FC0120836F5F862FF1
:100AC00090E09C01240F351F233831057CF381E031
:100AD00070CFEF92FF920F931F93DF93CF93CDB719
:100AE000DEB7A9970FB6F894DEBF0FBECDBFFC01ED
:100AF000DB018C918E32A9F1838590E08871907032
:100B00008031910509F466C0009759F5848D958D63
:100B1000A68DB78D803020E4920726E0A20720E062
:100B2000B20709F459C0803020E892072CE0A207F0
:100B300020E0B20709F454C0803020E8920726E193
:100B4000A20720E0B20709F449C081509044A640B2
:100B5000B0408F3F2FE2920721E1A20720E0B207C9
:100B600078F020E0822FA9960FB6F894DEBF0FBE72
:100B7000CDBFCF91DF911F910F91FF90EF9008951E
:100B8000CF017E010894E11CF11CB7010E94882866
:100B90001E86198A8E01025F1F4FC801B70141E00E
:100BA0000E94B32E882371F0C80163EC73E340E028
:100BB00052E00E944829C8010E94B22B809115344E
:100BC000813081F08989882361F2C8010E94B22BAB
:100BD00020E0C8CF21E0C6CF23E0C4CF25E0C2CFBC
:100BE00024E0C0CF80911634882361F780910434CB
:100BF00090E0A0E0B0E0BA2FA92F982F882720918D
:100C00000534820F911DA11DB11DB695A79597952D
:100C10008795B695A79597958795803921E0920796
:100C200020E0A20720E0B207F1F0803223E0920733
:100C300020E0A20720E0B207A1F0803A25E0920769
:100C400020E0A20720E0B20709F0BCCF28E08989A4
:100C5000882309F487CFC80129A70E94B22B29A5B0
:100C600081CF27E0F4CF26E0F2CF2F923F924F9230
:100C70005F926F927F928F929F92AF92BF92CF922C
:100C8000DF92EF92FF920F931F93DF93CF93CDB735
:100C9000DEB7C05FD0400FB6F894DEBF0FBECDBF49
:100CA0007C011092670310926603829640E050E048
:100CB000BA010E94CA2A03E4C02ED12CCC0EDD1E3C
:100CC00013E6A12EB12CAC0EBD1EB4E26B2E712C1E
:100CD000C701B601A50111DE8823E1F18091660309
:100CE0009091670321E08734920708F0A7C1C601FD
:100CF000B501EFDE882E882359F380916603909129
:100D00006703869D8001879D100D969D100D11240F
:100D10000D531C4FC801B50146E150E00E94393E19
:100D2000B8016A5E7F4FC6010E94882880916603E1
:100D300090916703869DF001879DF00D969DF00DC3
:100D40001124ED53FC4F83A2019690936703809387
:100D50006603BECF2091660330916703C751DF4F12
:100D600039832883C95ED040F70185A18250823043
:100D7000A8F184E290E0C751DF4FE881F981C95EB4
:100D8000D040E89F8001E99F100DF89F100D1124BD
:100D90000D531C4FC80160E071E046E150E00E9435
:100DA000393EC801469660E071E04DE050E00E9497
:100DB000393E82E0F80183A3C751DF4F2881398192
:100DC000C95ED0402F5F3F4FC751DF4F3983288323
:100DD000C95ED0403093670320936603A6EE2A2EA7
:100DE000A3E03A2E80E090E07E010894E11CF11C23
:100DF000F7E1CF2ED12CCC0EDD1EC751DF4FE8819D
:100E0000F981C95ED0408E179F0708F01EC1FC0112
:100E10003196C351DF4FF983E883CD5ED040C7518F
:100E2000DF4F28813981C95ED040E217F30708F00F
:100E300026C1C1018397F101B496C151DF4FF983F7
:100E4000E883CF5ED0405F01C351DF4F48805980B7
:100E5000CD5ED040CA51DF4F8883C65ED04091013D
:100E60002D503040C551DF4F39832883CB5ED040B1
:100E7000C951DF4F39822882C75ED040392EC70161
:100E8000CA51DF4F6881C65ED040732D46E150E005
:100E90000E94393E88240AC00E0D1F1DF801808172
:100EA00090E00E94FD3DF80180838394F70101905A
:100EB0000020E9F73197EE19FF09082D10E00E1711
:100EC0001F0750F3EDED8E2EEFEF9E2E8A0C9B1C2C
:100ED000682C292CC601B40146E150E00E94393E3D
:100EE00077240AC00C0D1D1DF801808190E00E943E
:100EF000FD3DF80180837394F60101900020E9F72D
:100F00003197EC19FD09072D10E00E171F0750F35C
:100F1000C701B60146E150E00E942B3E282F392F31
:100F2000C951DF4FE881F981C75ED040808181508F
:100F3000823008F480C0F50180818150823008F44D
:100F400077C0121613060CF055C0CE018D96CA510B
:100F5000DF4F6881C65ED040732D46E150E00E94AD
:100F6000393ECA51DF4F8881C65ED040932D662D31
:100F7000722D46E150E00E94393E862D922DBE0131
:100F8000635D7F4F46E150E00E94393ECE018D9671
:100F9000C551DF4F68817981CB5ED0404DE050E094
:100FA0000E94393E84010A5E1F4FC551DF4F888180
:100FB0009981CB5ED040B8014DE050E00E94393EAF
:100FC000C801BE01635D7F4F4DE050E00E94393E95
:100FD000C951DF4FE881F981C75ED0408081F501BA
:100FE0009081C951DF4FE881F981C75ED04090837D
:100FF000F50180830894411C511C24E230E0A20ECC
:10100000B31EC751DF4F88819981C95ED040481611
:10101000590608F434CFC151DF4F28803980CF5EA4
:10102000D040C351DF4F88819981CD5ED040E5CE5D
:1010300028513C4F86CF285E33407DCFC751DF4FCC
:1010400099838883C95ED0408FCEC051DF4F0FB6E1
:10105000F894DEBF0FBECDBFCF91DF911F910F91EE
:10106000FF90EF90DF90CF90BF90AF909F908F90C8
:101070007F906F905F904F903F902F900895C101A7
:101080008496C151DF4F99838883CF5ED040C3CF10
:101090008F929F92AF92BF92CF92DF92EF92FF9288
:1010A0000F931F93CF93DF9380916803909169030F
:1010B00020916A0330916B032817390728F4309385
:1010C000690320936803C90104968217930730F4DB
:1010D00024503040309369032093680380E060E03F
:1010E0000E94372281E06FE70E942822C3E1D0E00E
:1010F00081E060E40E9428222197D1F783E091E00B
:101100000E942C23C3E1D0E081E060E40E94282209
:101110002197D1F781E06FE70E9428222091660392
:10112000309167032115310509F464C140916803CA
:1011300050916903CA0105964817590708F033C151
:101140004217530708F02FC164E270E0469F700118
:10115000479FF00C569FF00C112486EE93E0E80EAA
:10116000F91EEA0191E0C92ED12CBB24B3948091E1
:101170006A0390916B03C817D90709F0BB24AC2C04
:1011800080E06C2D0E94372204E510E007C060E08B
:1011900081E00E9428220150104049F0BB20B9F3A1
:1011A0006FE781E00E94282201501040B9F781E0EA
:1011B0006A2D0E943722870103521040902E812E03
:1011C000C8016B2D43E50E944322F70180818150C5
:1011D000823008F4BDC0BB2009F0A4C0860121966E
:1011E0004091680350916903CA010596C817D90751
:1011F000E0F120916603309167032630310508F055
:1012000047C0EE24E39482E56E2D0E94372281E0F0
:1012100060E00E94282281E060E00E942822E3949E
:101220007E2D763081F78091680390916903980153
:10123000280F391F40916A0350916B0342175307DF
:1012400008F4E2C02150304030936B0320936A03CE
:101250000430110509F02CCF009709F429CF01972C
:10126000909369038093680323CF209166033091A4
:1012700067030894C11CD11C64E270E0E60EF71EFF
:10128000C217D30708F471CF2630310508F4B9CF5F
:10129000E7E2F0E04E9FC0014F9F900D5E9F900DE2
:1012A00011248D539F4FB9010E94A83D88E0E82E7C
:1012B000E60E83EC90E0B9010E94A83DCE2CC61A40
:1012C000C8E0D0E0BB24B39482E56B2D0E943722A6
:1012D00081E060E00E9428224C2F9E01295F3F4F51
:1012E0002C173D070CF484C060E00AC0E41650F0EF
:1012F000669560684F5F842F90E0281739074CF09F
:101300004C15A0F766954F5F842F90E0281739079A
:10131000BCF781E00E942822B39428967B2D76307A
:1013200099F681CF82E893E0692D782D46E150E06F
:101330000E94393EB8016A5E7F4F8CE693E04DE033
:1013400050E00E94393EF70180818093980346CF98
:1013500089E46A2D0E943722BB2041F181E06FE7CA
:101360000E94282281E063E40E94282281E06DE54A
:101370000E94282281E06DE50E94282281E06DE52F
:101380000E94282281E06BE50E94282281E06BE523
:101390000E94282281E063E40E9428226FE781E016
:1013A0000E94282218CF00E010E027CF81E060E003
:1013B0000E94282281E06CE30E94282281E062E200
:1013C0000E94282281E062E20E94282281E062E2FB
:1013D0000E94282281E064E20E94282281E064E2E7
:1013E0000E94282281E06CE30E94282260E0D7CF8F
:1013F00060E08FCF80E061E00E9437228FE091E0D3
:1014000060E044E50E944322DF91CF911F910F914C
:10141000FF90EF90DF90CF90BF90AF909F908F9014
:1014200008958130910559F0009721F48091EF35AE
:10143000882309F408958CEE95E30C94B22B109256
:10144000EC351092EF350895DF92EF92FF920F93F3
:101450001F93CF93DF93082F2B9882E282B95D9878
:10146000429A289A45980E947B23CDEAD3E0FE0158
:1014700001900020E9F73197EC1BFD0B8E2F819531
:10148000880F865D65E00E943722CE0160E044E56A
:101490000E9443220E94F021002309F438C00AE68A
:1014A00014E0DD2480E06D2D0E9437222AE1E22E37
:1014B00081E060E00E942822EA94D1F790E1E92ED1
:1014C000F12CE00EF11EE801FE01649181E00E9422
:1014D00028222196EC16FD06B9F7E8012F96015057
:1014E0001040FE01649181E00E94282221970C1790
:1014F0001D07B9F70AE181E060E00E94282201504F
:10150000D1F7D394FD2DF43051F18701CBCFC6E252
:10151000D4E0FF2480E06F2D0E94372201E281E0B9
:1015200060E00E9428220150D1F78E010F5E1F4F0C
:10153000FE01649181E00E94282221960C171D076C
:10154000B9F782E2E82E81E060E00E942822EA9466
:10155000D1F7F394FF2DF43011F0E801DBCF98E0E0
:101560002FEB37E249E0215030404040E1F700C026
:10157000000085B1892785B9F3CFEF920F9336B17B
:1015800091E0811190E0331F3327331F931759F0F7
:10159000E9B1E095E170F0E081E090E0662339F494
:1015A000E817F90749F080E00F91EF90089580E087
:1015B00090E0E817F907B9F766B16095617070E0DF
:1015C00081E090E0442311F080E090E06817790713
:1015D00051F790B181E0211180E0991F9927991F5F
:1015E000891709F326B191E0011190E081E021FF14
:1015F00080E09817C1F229B191E0E11090E081E01C
:1016000023FF80E08927D0CF559A209A3A9A3D9AB5
:101610003E9A3B9A239A289A429A45984698439A2A
:101620002B9A8FE781B95C9A599A5A9A5F9A5B9A7A
:10163000179A589A409A419AE3E7F0E080818160D6
:101640008083EDE6F0E0808182608083808181602C
:10165000808308951F93DF93CF93CDB7DEB72A978A
:101660000FB6F894DEBF0FBECDBFCE010196DC01F0
:10167000ECE2F3E02AE001900D922150E1F7E091D5
:101680009A03F0E0F595E795F595E795F595E795DB
:10169000F595E7951FB7F894E53008F0E4E0F0E041
:1016A000EE0FFF1FE80FF91F20813181220F331F3A
:1016B00040E050E060E07DE281E391E00E94DE3DA9
:1016C0003093A9032093A8031FBF82E086BB2A960C
:1016D0000FB6F894DEBF0FBECDBFCF91DF911F9143
:1016E00008951F920F920FB60F920BB60F9211240E
:1016F0002F933F934F935F936F937F938F939F931A
:10170000AF93BF93CF93DF93EF93FF93489B2FC08B
:10171000E0919A038091A303882309F03DC0F0E093
:10172000E45DFE4F249130E0220F331F2115310577
:10173000A9F537995DC080919A038F5F80939A03D2
:1017400080919A03882309F064C04598429A489989
:10175000FECF4298459A7EDFC091E235D091E335C5
:10176000C330D10508F057C081E080939F03FF91FB
:10177000EF91DF91CF91BF91AF919F918F917F9129
:101780006F915F914F913F912F910F900BBE0F90F2
:101790000FBE0F901F90189524E230E080E090E09B
:1017A00040E050E068E18A539A4CFC01808180FF60
:1017B00003C0683159F1542F4F5F842F90E0821796
:1017C00093070CF1561708F4B4CF862FE82FF0E0FA
:1017D000EA53FA4C908191FF03C09081916090830D
:1017E0009081946090838F5F581780F7379BA3CFC9
:1017F00080919A03882309F4A3CF80919A038150A2
:1018000080939A039DCF4831E9F2CDCF542F642FB6
:10181000D3CF459A9BCF8DEA93E061E371E046E137
:1018200050E00E94393EC851DC4FD093C535C0937B
:10183000C43510929E0381E080939F038093A003A0
:101840001092E3351092E2358FCF1F920F920FB6B0
:101850000F920BB60F9211241F932F933F934F9328
:101860005F936F937F938F939F93AF93BF93CF9328
:10187000DF93EF93FF9386B190E095958795817004
:1018800090919C03891791F09091A603923009F4EE
:101890006DC010929C0311E010939F03C091E2353C
:1018A000D091E335C330D10508F047C086B18170CF
:1018B00011E0812790919E038917C9F080939E03C0
:1018C00080919E03882349F546988FE781B98091DE
:1018D0006B008F7780936B00C091E235D091E33538
:1018E000C330D10508F045C081E080939F03FF918C
:1018F000EF91DF91CF91BF91AF919F918F917F91A8
:101900006F915F914F913F912F911F910F900BBE5F
:101910000F900FBE0F901F90189511B8469A8091A6
:101920006B00806880936B0080B180788093E13594
:101930001092E3351092E235D7CF8DEA93E061E360
:1019400071E046E150E00E94393EC053D84FD09339
:10195000C535C093C43510929E0310939F03109316
:10196000A0031092E3351092E235A0CF80939C0340
:1019700092CF8DEA93E061E371E046E150E00E948E
:10198000393EC854D44FD093C535C093C435109256
:101990009E0310939F031093A0031092E3351092BF
:1019A000E235A2CF1F93E0B1E0688091E2359091DB
:1019B000E3358430910588F48330910509F487C0BC
:1019C000DC01A35EBC4F2C912E1709F404C11092C8
:1019D000E3351092E2351F910895F0E0EA5DFE4F85
:1019E000E49132E08F3B930748F59C0123703070FF
:1019F0002230310509F4BBC02330310509F449C157
:101A00002130310509F418C1EE0FEE0FE093E435F3
:101A10004091E83550E09A01220F232F221F330B0B
:101A20002093E935440F551F422B4093E83501962A
:101A30009093E3358093E2351F910895F2E08F3B58
:101A40009F0709F4C1C022E0803C920709F4CEC090
:101A500032E0813C930709F4E2C1F2E0823C9F0747
:101A600009F0B5CF8091E435982F990F990F909395
:101A7000E435E82B9091E835E917C9F08DEA93E059
:101A800062E971E046E150E00E94393E80E490E076
:101A90009093C5358093C43510929E0381E0809366
:101AA0009F038093A0031092E3351092E235E091FA
:101AB000E535F0E0EA53FA4C8081826080838081D2
:101AC0008160808380818B7F80832B9A80CFF0E040
:101AD000EA5DFE4F1491E0919A038091A30388235D
:101AE00009F082C0F0E0E45DFE4FE4911E1708F0BB
:101AF0004DC1E0919A03882309F074C0F0E0E45DE1
:101B0000FE4FE49180919C03E89F802D1124810F6A
:101B10008093E53590E0DC01AA53BA4C2C9122FD6C
:101B2000E0C0982F8827990F8D539C4F9093EB35E9
:101B30008093EA358C9184608C938C918D7F8C930B
:101B400080919A038093DE3580919C038093DF35EA
:101B50001093E0352B981092E8351092E7351092EB
:101B6000E6358091E2359091E335019661CF509151
:101B7000E435452F407C4E2B2091E63542278431B9
:101B8000910578F0E091EA35F091EB354193F093CF
:101B9000EB35E093EA355091E4358091E235909150
:101BA000E3356091E9352091E73530E0260F311DAE
:101BB000240F311D2093E7353093E935550F550F2C
:101BC0005093E435019634CFEE0FEE0FE093E435F9
:101BD00080EC92E02DCF2091A203222309F0F7CED2
:101BE000019626CFE2E18ECFE2E180CF8091E4350D
:101BF000982F990F990F9093E435807C8E2B9091BC
:101C0000E635891709F46AC08DEA93E06CE671E065
:101C100046E150E00E94393E8EE390E09093C53556
:101C20008093C43510929E0381E080939F0380933C
:101C3000A00381E090E0FCCE5091E435452F407C3C
:101C40004E2B2091E83542278431910578F0E091C0
:101C5000EA35F091EB354193F093EB35E093EA35BB
:101C60005091E4358091E2359091E3356091E9350A
:101C70002091E63530E0260F311D240F311D2093D1
:101C8000E6353093E935550F550F5093E4350196FD
:101C9000CFCE4091E4354E2B2091E7354227843159
:101CA000910568F0E091EA35F091EB354193F093BE
:101CB000EB35E093EA358091E2359091E335509130
:101CC000E9352091E83530E0250F311D240F311D15
:101CD0002093E8353093E9350196AACE81EC92E065
:101CE000A7CE30919A0320919C038DB79EB70C9795
:101CF0000FB6F8949EBF0FBE8DBFADB7BEB711969D
:101D00008DEA93E0EDB7FEB79283818386E190E0A0
:101D100013969C938E93129788E591E015969C9369
:101D20008E93149716963C93169717961C921797B6
:101D300018962C93189719961C9219971A961C931B
:101D40001A971B961C920E94483E8DE390E0909358
:101D5000C5358093C43510929E0381E080939F0324
:101D60008093A0031092E3351092E2358091E5351F
:101D700090E02DB73EB7245F3F4F0FB6F8943EBFBB
:101D80000FBE2DBFDC01AA53BA4CCBCE20919A03D3
:101D90008DB79EB70A970FB6F8949EBF0FBE8DBF42
:101DA000ADB7BEB711968DEA93E0EDB7FEB792835B
:101DB000818386E190E013969C938E93129782E440
:101DC00091E015969C938E93149716961C931697F4
:101DD00017961C92179718962C93189719961C9281
:101DE0000E94483E8CE390E09093C5358093C435C3
:101DF00010929E0381E080939F038093A003109232
:101E0000E3351092E2358091A3032DB73EB7265FEC
:101E10003F4F0FB6F8943EBF0FBE2DBF6ACE8091E4
:101E2000E435982F990F990F9093E435807C8E2B91
:101E30009091E735891759F08DEA93E06FE771E0EB
:101E400046E150E00E94393E8FE390E0E7CE82EC1D
:101E500092E0EECD4091A4035091A503E2EEF2E0B2
:101E60002591349160E07FEF2627372791EA692F8B
:101E7000632770E0660F771F6A5D7D4FFB016591F8
:101E80007491322F2227262737279327E92FF0E056
:101E9000EE0FFF1FEA5DFD4F65917491322F2227EF
:101EA00026273727EBEFE327F0E0EE0FFF1FEA5D71
:101EB000FD4F65917491322F222726273727B82F9F
:101EC000BB0FA0E0AD53BC4F80E090E0722F6627BF
:101ED000ED91E327F0E0EE0FFF1FEA5DFD4F259146
:101EE000349126273727019662E08030960771F7F4
:101EF0003093A5032093A40342175307C9F08DEA3A
:101F000093E065EA71E046E150E00E94393E86E4E4
:101F100090E09093C5358093C43510929E0381E084
:101F200080939F038093A0031092E3351092E235D3
:101F300008951F920F920FB60F920BB60F921124B5
:101F40002F933F934F935F936F937F938F939F93C1
:101F5000AF93BF93EF93FF9390B180919E0388233B
:101F600009F456C0892F80789091E135891709F4DA
:101F70004FC08093E1359091A303992309F46FC07A
:101F8000882309F461C020B12F708091E435282B9B
:101F90002093E4358091E2359091E33582309105CC
:101FA00009F45FC0009709F446C08130910509F437
:101FB0006DC032E08330930708F458C0A2E083304C
:101FC0009A0709F49AC0B2E084309B0709F530E023
:101FD0008091A4039091A503822B932B9093A5034A
:101FE0008093A4038091E53535DFE091E535F0E09D
:101FF000EA53FA4C80818260808380818160808393
:1020000080818B7F80832B9A1092E3351092E2358A
:10201000FF91EF91BF91AF919F918F917F916F91C0
:102020005F914F913F912F910F900BBE0F900FBE7C
:102030000F901F901895213A59F781E090E0909306
:10204000E3358093E235E4CF80B190E082959295BC
:10205000907F9827807F98278093E435D9CFA2DCA2
:10206000D7CF2B3FE9F0213A79F6D2CF3091E53541
:10207000F32FFF0FE0E0E80FF91FE054FC4F20833F
:1020800001969093E3358093E235C2CF213A09F06F
:10209000BBCF82E090E09093E3358093E235B8CFF8
:1020A00083E090E09093E3358093E2352091A7039D
:1020B0002093E535822F90E0FC01EA53FA4C308101
:1020C00032FD26C0982F8827990F8D539C4F9093EF
:1020D000EB358093EA3580818460808380818D7FB9
:1020E000808380919A038093DE3580919C03809356
:1020F000DF352093E0352B988BCF1092A4032093EB
:10210000A50384E092E09093E3358093E23580CF9D
:1021100050919A0340919C032DB73EB72C5030400C
:102120000FB6F8943EBF0FBE2DBFEDB7FEB7319688
:102130002DEA33E0ADB7BEB712963C932E931197BC
:1021400026E130E03383228328E531E035832483A0
:102150005683178240871186938782870E94483E64
:1021600087E490E09093C5358093C43510929E0328
:1021700081E080939F038093A0031092E335109237
:10218000E2352DB73EB7245F3F4F0FB6F8943EBF00
:102190000FBE2DBF3DCFF89490919E03992341F43B
:1021A0008F7782B9459A079BFECF0799FECF459856
:1021B000789408958AE082B9459A079BFECF0799E3
:1021C000FECF4598E091A50381EAE827F0E0EE0F05
:1021D000FF1FEA5DFD4F859194913091A40320E0AB
:1021E000822793279093A5038093A40381E182B96A
:1021F000459A079BFECF0799FECF45980895982FE3
:1022000092959F7092B9459A079BFECF0799FECF92
:102210004598482F4F70E091A503E827F0E0EE0FB6
:10222000FF1FEA5DFD4F859194913091A40320E05A
:10223000822793279093A5038093A40342B9459ADC
:10224000079BFECF0799FECF459808952F923F92A6
:102250004F925F926F927F928F929F92AF92BF92B6
:10226000CF92DF92EF92FF920F931F93DF93CF9362
:1022700000D00F92CDB7DEB78983692EA0E2CA2EB7
:10228000A3E0DA2E992422243324EE24FF2400E054
:1022900010E088C01070C801880F991F2801440CF5
:1022A000452C441C55085194482A592AF60101919D
:1022B000852D9927820D931D800F911DAFEF4A2226
:1022C0005524D6011196AC906F010894C11CD11C05
:1022D000A7014A0D511D9C0120703170232F332717
:1022E000420F531F3FEF232E312C282239227180B9
:1022F0002FEFE22EF12CE422F522872C8E240425E8
:1023000010E0A224BB24F501E07CF070F595E79580
:10231000F595E795F595E795F595E7959801207C76
:1023200030703595279535952795E22BF32B882D21
:10233000829586958695837090E0E82BF92BE4587A
:10234000FE4F84914A835B8326DF0F73107004581D
:102350001E4FF80184911FDF80919F034A815B81AA
:10236000882309F0A9C00894C11CD11C8201070D63
:10237000111D40705170452F5527040F151FF50191
:10238000EF73F070E458FE4F849105DFE82DF0E024
:10239000EF73F070E458FE4F8491FDDE9394F92DB5
:1023A000FE3A41F0292D243009F074CF9981C92ECD
:1023B000D62C70CF1070C801880F991F5801AA0C35
:1023C000AB2CAA1CBB08B194A82AB92AD6010C913F
:1023D000200E311C8B2D9927280E391E1196CC907A
:1023E000EC0CF11CC10180709170892F9927E80EC7
:1023F000F91E0A2510E0C224DD24F601E07CF0700D
:10240000F595E795F595E795F595E795F595E795B4
:10241000C801807C90709595879595958795E82B58
:10242000F92BE458FE4F8491B6DEF801EF73F0709B
:10243000E458FE4F8491AFDEF601EF73F070E4587C
:10244000FE4F8491A8DEF101E07CF070F695E795EF
:10245000F695E795C501807C90700024880F991F40
:10246000001C880F991F001C892F902DE82BF92B39
:10247000C701807C9070929582958F7089279F709C
:102480008927E82BF92BE458FE4F849184DEF10173
:10249000EF73F070E458FE4F84917DDEF701EF7327
:1024A000F070E458FE4F849176DEF501EF73F07022
:1024B000E458FE4F84916FDE0F900F900F90CF91F4
:1024C000DF911F910F91FF90EF90DF90CF90BF9021
:1024D000AF909F908F907F906F905F904F903F90C4
:1024E0002F9008951F93CF93DF938FEF99E6A8E184
:1024F00081509040A040E1F700C000008CEE95E3D1
:1025000063EB71E041E00E94B32E882309F46DC0B3
:102510008CEE95E363EC73E040E052E00E944829C2
:1025200097FD78C010920836109207368BE796E137
:102530000E94483D1FB7F8940E94F23CEC011FBF77
:102540008CEE95E30E94B22B0E946F23209761F1DD
:10255000ADB7BEB718970FB6F894BEBF0FBEADBFEC
:10256000EDB7FEB731968DEA93E012969C938E9369
:10257000119786E190E09383828380ED91E09583CB
:102580008483D783C6830E94483E8DB79EB7089642
:102590000FB6F8949EBF0FBE8DBF81E00E94240A43
:1025A000DF91CF911F91089589E062E00E94372268
:1025B0008DEA93E060EC71E046E150E00E94393E24
:1025C0008DEA93E060E044E50E9443228FEF9AE1B8
:1025D000A7EB81509040A040E1F700C00000FE0151
:1025E0000995DF91CF911F91089564E00E943722F1
:1025F0008BE696E060E00E94C4228DEA93E06EE5EF
:1026000076E00E94053E80E00E94240ADF91CF918F
:102610001F9108958DEA93E06EE476E00E94053EF6
:1026200081E00E94240A7ECFCF93DF930E946F2324
:1026300080E060E00E94372288E396E061E00E943B
:10264000C42286E296E00E940C3E8195880F865D4A
:1026500062E00E94372286E296E060E00E94C42297
:102660004DB75EB7485050400FB6F8945EBF0FBEEE
:102670004DBFEDB7FEB73196CDEAD3E0ADB7BEB7EB
:102680001296DC93CE93119786E190E09383828338
:1026900082EE91E0958384838091AC0386831782D8
:1026A0000E94483EFE0101900020E9F73197EC1BA3
:1026B000FD0B4DB75EB7485F5F4F0FB6F8945EBF36
:1026C0000FBE4DBF8E2F8195880F865D63E00E94FF
:1026D0003722CE0160E044E50E9443220E94F021AF
:1026E00093E028E04FEF53ED60E3415050406040ED
:1026F000E1F700C0000085B1822785B9915091F7BC
:102700000E94F421DF91CF910895CF92DF92EF9252
:10271000FF920F931F93DF93CF9300D000D0CDB7DC
:10272000DEB780E060E00E9437220E946F2380E0E5
:1027300060E00E94372282E196E060E00E94C422BD
:1027400080E062E00E9437228FEF95E060E00E9417
:10275000C42280E063E00E94372289EF95E060E0C8
:102760000E94C422499BFECF4A9BFCCF4C9BFACFD0
:1027700080E060E00E9437220E946F2380E062E0E8
:102780000E9437228BEE95E060E00E94C42280E038
:1027900063E00E9437228EED95E060E00E94C42243
:1027A00080E064E00E94372281ED95E060E00E94C5
:1027B000C4228E010F5F1F4F83EFE82E81E0F82EB9
:1027C000B4E0CB2ED12C16C0809115368F3F29F066
:1027D000809115368F5F8093153680E061E20E940C
:1027E00028226091153680E00E94282280E060E275
:1027F0000E94282280E060E00E94372286EC95E06B
:1028000060E00E94C422809115362DB73EB7285053
:1028100030400FB6F8943EBF0FBE2DBFEDB7FEB7E8
:102820003196ADB7BEB712961C930E931197D38213
:10283000C282F582E482868317820E94483E2DB7C9
:102840003EB7285F3F4F0FB6F8943EBF0FBE2DBF77
:10285000C80160E044E50E9443228FEF99E6A8E1B9
:1028600081509040A040E1F700C00000499B04C0A7
:102870004A9B02C04C99FACF4A9BA6CF49990BC0FC
:1028800080911536813808F4A8CF80911536815093
:1028900080931536A2CF4C99A0CF6091153681E078
:1028A00090E00E9490408FEF99E6A8E1815090401F
:1028B000A040E1F700C000000E946F230F900F902E
:1028C0000F900F90CF91DF911F910F91FF90EF909C
:1028D000DF90CF90089580E060E00E9437220E9450
:1028E0006F2380E060E00E94372280EB95E061E09A
:1028F0000E94C42289E062E00E94372280EA95E0CB
:1029000060E00E94C42289E063E00E94372280E9EF
:1029100095E060E00E94C4228FE065E00E943722CB
:1029200084E895E060E00E94C422DCCD1F930E9401
:102930006F2380E060E00E94372282E893E060E04D
:1029400044E50E94432280E061E00E9437228CEE41
:1029500095E36CE673E043E00E94B32E882309F40C
:102960008AC080919803833029F1863019F182E082
:102970008093A6038CEE95E369E076E34DE056E3A1
:102980000E94D5278823D1F48BE595E060E00E9472
:10299000C4228FEF93E2A4EF81509040A040E1F772
:1029A00000C0000010E08CEE95E30E94B22B812F56
:1029B0001F91089581E08093A603DCCF80E061E061
:1029C0000E94372280919803853009F4BFC0863079
:1029D00008F05FC0833009F4A1C0843039F48DE37E
:1029E00095E060E00E94C4228091980391E08630D7
:1029F00008F490E09093C3354F998CC0992309F463
:102A00005CC081E08093A20348E754E060E070E09E
:102A10008CEE95E30E94CA2A8CEE95E363EC73E09A
:102A200040E052E00E944829E091C303F0E0EC53FB
:102A3000FC4F10821092D90380E062E00E9437229E
:102A400084EC93E060E044E50E94432280E064E08F
:102A50000E94372282EE94E060E00E94C4228091BE
:102A6000A203882379F511E08CEE95E30E94B22B46
:102A7000812F1F9108958CEE95E36CE673E041E0A1
:102A80000E94B32E882309F464C081E08093A203DE
:102A900071CF873009F452C0873008F447C08830BE
:102AA00009F0A4CF80EF94E060E00E94C42281E0AE
:102AB0008093A3038091980399CF44E254E060E0AF
:102AC00070E0A6CF8DE460E00E94372281E060E0F4
:102AD0000E94282281E068E70E94282281E06EE7B8
:102AE0000E94282281E069E70E94282281E069E7AC
:102AF0000E94282281E06EE70E94282281E068E798
:102B00000E94282211E08CEE95E30E94B22B812FC7
:102B10001F91089581E08093A20370CF8CE495E02B
:102B200060E00E94C4228091980360CF89E195E023
:102B300060E00E94C4228091980358CF85E095E020
:102B400060E00E94C4228091980350CF8DE295E00E
:102B5000ABCF80E795E060E00E94C4221ACF2898AE
:102B60008FE798E3A1E081509040A040E1F700C0DA
:102B7000000082E282B95D98289A0C947B231F930F
:102B80001FB7F894E0919A03F0E0EE0FFF1FE850B2
:102B9000F041808180939A030E94040B10929A0363
:102BA00010929B0310929F0310929C0310929D031E
:102BB00010929E031092A10382E08093A6031092CC
:102BC000A7031092A2031092A3031092A0031092E5
:102BD000AB031092AA031092C5351092C43510921F
:102BE000E3351092E23580E090E0FC01EA53FA4CC4
:102BF0001082019688319105C1F711B8469A28983C
:102C00008FE798E3A1E081509040A040E1F700C039
:102C1000000080B18F778093AC0346988FE781B92D
:102C2000289A9DDF0E946F231FBF1F910895FF9276
:102C30000F931F93CF93DF938C01F090A003C0916B
:102C4000C435D091C5359BDF0E946F2380E060E0E2
:102C50000E943722FF2009F43FC082E597E061E03F
:102C60000E94C42280E061E00E943722C80160E037
:102C700044E50E9443228DB79EB708970FB6F8949B
:102C80009EBF0FBE8DBFEDB7FEB731960DEA13E0C4
:102C9000ADB7BEB712961C930E93119786E190E0E4
:102CA0009383828386EF91E095838483D783C68361
:102CB0000E94483E8DB79EB708960FB6F8949EBF07
:102CC0000FBE8DBF80E065E00E943722C80160E042
:102CD00044E50E944322FFCF8CE397E061E00E942D
:102CE000C42280E061E00E943722C80160E044E530
:102CF0000E944322F0CF209107363091083682E0BF
:102D00002030380759F0F901ED53FC4F80812F5FD7
:102D10003F4F309308362093073608958CEE95E3A5
:102D200063EC73E040E052E00E94482997FD0BC03D
:102D3000109208361092073685B198E0892785B938
:102D400020E030E0E0CF89EF91E071DFF1CF9F929A
:102D5000AF92BF92CF92DF92EF92FF920F931F93A9
:102D6000CF93DF9387E893E10197F1F700C000006C
:102D700029E0E0E0F0E0209357006491A7E8B3E198
:102D80001197F1F700C00000E3E0F0E02093570056
:102D9000849190E0E7E8F3E13197F1F700C000009B
:102DA000E2E0F0E020935700249130E0A7E8B3E19F
:102DB0001197F1F700C000008A3D910509F418C28F
:102DC000EDB7FEB73C970FB6F894FEBF0FBEEDBF50
:102DD00031967DEAC72E73E0D72EADB7BEB71296F7
:102DE000DC92CE92119746E150E05383428349E052
:102DF00052E05583448366831782918780873387A7
:102E000022870E94483EEDB7FEB73C960FB6F89475
:102E1000FEBF0FBEEDBF81E00E94240A2091AC03EB
:102E20002F3709F4F2C12D3049F14DB75EB7485044
:102E300050400FB6F8945EBF0FBE4DBFEDB7FEB762
:102E40003196ADB7BEB71296DC92CE92119786E15D
:102E500090E09383828380E392E09583848326834A
:102E600017820E94483EEDB7FEB738960FB6F89429
:102E7000FEBF0FBEEDBF81E00E94240A10928000C9
:102E8000109281008091640088608093640028988B
:102E900012B842985D98459881E061E041E021E0F8
:102EA00000E0EE240E94BD0A882309F420C211E04C
:102EB00012B980E061E041E021E000E0EE240E94F0
:102EC000BD0A8127C82FD0E012B8429A81E061E0A4
:102ED00041E021E00E94BD0AF82E12B981E061E0D4
:102EE00041E021E00E94BD0AF1262F2D30E02C2B7D
:102EF0003D2B1827122B09F0F0C112B8429852E06E
:102F0000F52EF2B8A12EBB2481E060E041E021E083
:102F100000E0EE240E94BD0A982E12B85D9A81E06E
:102F200061E041E021E00E94BD0A11E09126C92D37
:102F3000D0E0812790E0C82BD92BF2B881E061E086
:102F400041E021E00E94BD0ACA29DB2918271C2B79
:102F500009F0B9C112B85D9844E0F42EF2B8A12E80
:102F6000BB2481E061E040E021E000E0EE240E942B
:102F7000BD0A982E12B8459A81E061E041E021E057
:102F80000E94BD0A11E09126C92DD0E0812790E072
:102F9000C82BD92BF2B881E061E041E021E00E942A
:102FA000BD0ACA29DB2918271C2B09F082C112B8D7
:102FB000459880E282B9A12EBB2481E061E041E026
:102FC00020E000E0EE240E94BD0AF82E88E082B9DD
:102FD00081E061E041E021E00E94BD0A11E0F126BC
:102FE000CF2DD0E0812790E0C82BD92B88E282B981
:102FF00081E061E041E021E00E94BD0ACA29DB29AD
:1030000018271C2B09F04BC112B880E182B981E06E
:1030100061E041E021E001E0EE240E94BD0AFF24CE
:10302000F394F826F12A09F030C112B880E482B98D
:1030300081E061E041E021E000E0EE24E3940E94C1
:10304000BD0A91E09827892F90E02F2D30E0822B48
:10305000932B009709F00FC112B8289A90DD489978
:1030600000C1459A11B8469A8FEF9FEF03C00197B0
:1030700009F447C1079BFBCF8FEF9FEF03C0019778
:1030800009F449C10799FBCF459846988FE781B964
:1030900081E060E041E020E000E0EE240E94BD0A13
:1030A000882309F4D4C00AE614E0AA2480E06A2D3B
:1030B0000E9437223AE1F32E81E060E00E9428224C
:1030C000FA94D1F7F02EE12EC0E0D0E00DC0C70198
:1030D000E92FFE2DEC0FFD1F649181E00E94282254
:1030E0002196C031D10531F09A2D923081F7EAEA6C
:1030F000F4E0F0CFCFE0D0E00EC0C701E92FFE2D05
:10310000EC0FFD1F649181E00E9428222197BFEF00
:10311000CF3FDB0731F0AA2DA23079F7EAEAF4E0DD
:10312000EFCF2AE1F22E81E060E00E942822FA949B
:10313000D1F7A394005F1F4FEA2DE43009F0B6CF1A
:1031400000D000D000D0EDB7FEB73196ADB7BEB716
:103150001296DC92CE92119786E190E0938382835F
:1031600080E492E0958384830E94483EF6010190BA
:103170000020E9F73197ED5AF3402DB73EB72A5FAB
:103180003F4F0FB6F8943EBF0FBE2DBF8E2F8195D7
:10319000880F865D65E00E943722C60160E044E545
:1031A0000E9443222B988FEF93EDA0E38150904033
:1031B000A040E1F700C0000085B198E0892785B9FB
:1031C0002FEF33ED40E3215030404040E1F700C0A5
:1031D000000085B1892785B9DF91CF911F910F91AB
:1031E000FF90EF90DF90CF90BF90AF909F900895A9
:1031F0002C3F310509F0E4CDEDEACE2EE3E0DE2EE2
:103200002091AC032F3709F00ECE00D000D000D0B3
:10321000EDB7FEB73196ADB7BEB71296DC92CE923F
:10322000119786E190E09383828382E292E0958316
:1032300084830E94483EEDB7FEB736960FB6F894E9
:10324000FEBF0FBEEDBF80E00E94240A17CE8DEABC
:1032500093E06AE776E00E94053E81E00E94240A3E
:1032600022CF8DEA93E061EB76E00E94053E81E09B
:103270000E94240AF6CE8DEA93E061EC76E00E948B
:10328000053E81E00E94240AE7CE8DEA93E061EDDD
:1032900076E00E94053E81E00E94240AC6CE8DEAB7
:1032A00093E065EE76E00E94053E81E00E94240AEC
:1032B000ABCE8DEA93E066EF76E00E94053E81E0BA
:1032C0000E94240A74CE8DEA93E065E077E00E94C4
:1032D000053E81E00E94240A3DCE8DEA93E068E13C
:1032E00077E00E94053E81E00E94240A06CE8DEA26
:1032F00093E06BE277E00E94053E81E00E94240AA1
:10330000D6CD8DEA93E060EA76E00E94053E81E04A
:103310000E94240AB1CE8DEA93E06FE876E00E9425
:10332000053E81E00E94240AAFCEE4E6F0E0808111
:10333000877F808383E48093800089E1809381008C
:103340000C942A0B9091A3039923E1F4E82FF0E069
:10335000E45DFE4FE491F0E0262F30E02E173F07AA
:10336000B4F4AF014F5F5F4F55954795E0FD14C032
:1033700031972E173F0759F06417B0F0862F8F5FF3
:10338000841B0895262F30E02131310514F080E0B0
:103390000895862F8F5F0895E42FF0E031972E1760
:1033A0003F0751F780E00895842F860F0895FF921C
:1033B0000F931F938C01F22E0E94D424882379F15D
:1033C000C80163EC73E30E942C24882391F1E7E1A8
:1033D000F4E3BF2DBB0FA0E0AD53BC4F81918D93A3
:1033E00085E3E33CF807D1F7C80163EC73E30E947F
:1033F0002C24882311F1E3ECF3E3BF2DBB0FA0E0F5
:10340000A159BA4F81918D9384E3E731F807D1F741
:10341000C8010E94BC241F910F91FF9008958DE474
:1034200092E005DCC80163EC73E30E942C2488233E
:1034300071F681E692E0FBDBCACF81E692E0F7DB32
:10344000DACF2F923F924F925F927F928F929F920C
:10345000AF92BF92CF92DF92EF92FF920F931F93A2
:10346000DF93CF93CDB7DEB760970FB6F894DEBF8A
:103470000FBECDBF982E792E862E8091A303882370
:1034800009F4B7C004E210E0F2E14F2E512C80E0C5
:1034900090E020E0FF24E8E1EE2E76E1A72EB12CAB
:1034A00061E7C62E62E0D62E1801122F8A539A4C7D
:1034B000DC018C9180FF35C08091DE35881661F18A
:1034C0008091DE352DB73EB72A5030400FB6F894C4
:1034D0003EBF0FBE2DBFEDB7FEB731962DEA33E0EC
:1034E000ADB7BEB712963C932E931197B382A282CA
:1034F000D582C48286821782808711860E94483EC8
:103500004DB75EB7465F5F4F0FB6F8945EBF0FBE14
:103510004DBF8DEA93E08BDB5E2D583109F466C018
:10352000F12E1F5F812F90E0821593050CF45AC095
:10353000BE2DB83109F43EC08091A203882361F406
:1035400066C0EE2DF0E0EA53FA4C80818E7F8083D6
:1035500080818B7F8083E394FE1498F7EDB7FEB7EC
:1035600038970FB6F894FEBF0FBEEDBF31960DEA47
:1035700013E0ADB7BEB712961C930E93119786E178
:1035800090E09383828386E892E0958384838682A9
:1035900017820E94483EEDB7FEB738960FB6F894F2
:1035A000FEBF0FBEEDBF80E065E061D7C80160E0FF
:1035B00044E569D760960FB6F894DEBF0FBECDBF65
:1035C000CF91DF911F910F91FF90EF90DF90CF90FF
:1035D000BF90AF909F908F907F905F904F903F9063
:1035E0002F900895183109F4A3CF60CFF12EE12E6A
:1035F00098CFE62FF0E0E45DFE4FE4914E2E552487
:103600008201000F111F01151105A1F240CFE8D66C
:1036100013D76B877C878D879E87FE1408F461C162
:10362000482D50E05A8749871A01220C331CC101EA
:10363000880F991F880F991F880F991F820D931D5E
:103640009C0140E050E029833A834B835C830E2D3C
:10365000F101E457FF4F859194919C0140E050E0C7
:103660002D833E834F8358871E2DAF2C42C0809000
:10367000DF352091A60330E040E050E069817A8197
:103680008B819C810E94893D6B017C018091093670
:1036900090910A36A0910B36B0910C36C80ED91E07
:1036A000EA1EFB1E282D30E0429EC001439E900D75
:1036B000529E900D1124AA2797FDA095BA2FC80EEF
:1036C000D91EEA1EFB1EC00ED11CE11CF11C2F8569
:1036D0003889322F2227330F2D533C4F892D972DB8
:1036E000B701A6010E94F424882371F10F5FA01690
:1036F00088F1402F50E0588B4F87FA01EA53FA4C7B
:10370000808180FDF3CF8091A303882309F0AFCFA0
:10371000C0900936D0900A36E0900B36F0900C3607
:10372000C00ED11CE11CF11C2091A60330E040E04A
:1037300050E06D817E818F8198850E94893DC60E03
:10374000D71EE81EF91EC3CF8BE992E070DA0F5F37
:10375000A01678F6E12EFA2C8091A303882309F0B5
:103760004FC0F101E457FF4F65917491A090093665
:10377000B0900A36C0900B36D0900C36AE0CB11C0F
:10378000C11CD11C80E090E02091A60330E040E015
:1037900050E00E94893DA60EB71EC81ED91E0F2DEF
:1037A00010E00F5F1F4F0E191109222717FD2095FA
:1037B000322F892D972DB601A5010E948F268823CF
:1037C00059F487C0F801EA53FA4C80818E7F8083D8
:1037D00080818B7F8083E394FE14D0F10E2D10E066
:1037E000B801762F6627770F6D537C4F892D972D63
:1037F0000E941D26882331F78EEB92E018DAE2CF83
:103800008091DF3590E0489E5001499EB00C589E53
:10381000B00C1124CC24B7FCC094DC2C8091093668
:1038200090910A36A0910B36B0910C36A80EB91EB5
:10383000CA1EDB1EAE0CB11CC11CD11CB101660F2F
:10384000771F660F771F660F771F620D731D9ACF64
:10385000892D972D0E94D026882309F43EC089E146
:103860008093AB03C1D5E8D5ADB7BEB71C970FB6F3
:10387000F894BEBF0FBEADBFEDB7FEB731960DEAEF
:1038800013E012961C930E93119726E130E03383D8
:1038900022832FED32E03583248329853A853783CF
:1038A00026832B853C854D855E85621B730B840BBF
:1038B000950B60877187828793870E94483E4DB73A
:1038C0005EB7445F5F4F0FB6F8945EBF0FBE4DBF4B
:1038D0006ACE8BEA92E0ABD97FCF8DEC92E0A7D98C
:1038E000BECF282D30E03A8729871901220C331CDE
:1038F00033CF2F923F924F925F926F927F928F922F
:103900009F92AF92BF92CF92DF92EF92FF920F936E
:103910001F93DF93CF93CDB7DEB7CD54D0400FB612
:10392000F894DEBF0FBECDBF55D529D9499B04C041
:103930004A9902C04C9B07C0499904C04A9902C0E9
:103940004C9901C004DAF1DC0E941413C8D67894B3
:103950008FE79AE1A6E081509040A040E1F700C0D7
:1039600000003ED58FE79AE1A6E081509040A0404C
:10397000E1F700C00000499B06C04A9904C04C9979
:1039800002C00E94851389E189831C821C8E1BA2C0
:103990001EA28E010F5F1F4FC80161E00E94352FEC
:1039A000882309F49BC45DEA852E53E0952E1CD52F
:1039B000499906C04A9904C04C9B02C00E946B14EE
:1039C000C8010E943506C8010E94480822243324F9
:1039D0008091A003882309F078C0F894D0909A03CE
:1039E000C0909C0310929F0378948091A103882338
:1039F00009F07EC080919F03882351F74B9B04C040
:103A000007996DC0F1010995499918C080916A0321
:103A100090916B03009771F3019790936B038093E0
:103A20006A03C8010E9448088FEF94E3ACE081501C
:103A30009040A040E1F700C00000DCCF4A9B49C0A5
:103A40004C99D8CF80919803813009F405C3823016
:103A500009F499C280916800886080936800809121
:103A6000680084608093680080916800846080931F
:103A700068008091680081608093680010929A03CA
:103A80002ED60E949614882309F4A2CF8091A20317
:103A900091E089279091A303992309F4826082B968
:103AA000459AA7E8B3E11197F1F700C000004598E7
:103AB000B2E4BA95F1F700C04298E1E0E093A103C7
:103AC0008091A003882309F488CF8DEA93E0AFD8D2
:103AD00084CF80916A0390916B0301969ECF89B148
:103AE00080FF90CF86B180FF8DCF31998DCF8ACF67
:103AF000ED2CFF242DB73EB7285030400FB6F89478
:103B00003EBF0FBE2DBFEDB7FEB73196ADB7BEB706
:103B100012969C928E92119726E1422E512C53823E
:103B2000428294E1692E93E0792E75826482F78255
:103B3000E6820E94483E2DB73EB7285F3F4F0FB642
:103B4000F8943EBF0FBE2DBF88E164E090D4C4015D
:103B500060E044E598D4AC2CBB248DB79EB70897A1
:103B60000FB6F8949EBF0FBE8DBFEDB7FEB731966E
:103B7000ADB7BEB712969C928E9211975382428235
:103B800089E1482E83E0582E55824482B782A6826E
:103B90000E94483E2DB73EB7285F3F4F0FB6F894BE
:103BA0003EBF0FBE2DBF88E364E061D4C40160E076
:103BB00044E569D480919B038D1509F4BDC16091E2
:103BC0009B03C8013EDCD0929B03C0929D0380E022
:103BD00090E0FC01EA53FA4C20812D7F208301966E
:103BE00088319105B1F780919F03882309F0F0CEC9
:103BF00080919E03882309F091C13D2D303598F7BF
:103C00008091A303882309F0BCC1F701E45DFE4F56
:103C100024918091A703821710F01092A70386B118
:103C20004B9903C3881F8827881F8EAF2C9D902D2A
:103C3000112423969FAF2397A701440F551FCA0154
:103C4000880F991F880F991F880F991F840F951F40
:103C500028968FAF289729969FAF299730E02A9D05
:103C6000C0012B9D900D3A9D900D11242C016624CE
:103C700057FC6094762C27964CAE5DAE6EAE7FAE50
:103C800027970E2CEF2C000CEE1CFF08000CEE1CEE
:103C9000FF1CAA0CBB1CA294B294E0EFBE22BA2473
:103CA000AE22BA245E2C5A285FAE852D90E084584F
:103CB0009E4F44575F4FFA01659074902B967FAEEC
:103CC0006EAE2B972D2D2F7321962FAF2197E22FBC
:103CD000F0E0E458FE4F34912C963FAF2C97FC0156
:103CE000F4912D96FFAF2D972296DFAE22972E9658
:103CF000CFAE2E972401F6B0F094FF1CFF24FF1CDA
:103D000009F474C16EAC6F1461F080E464E0AFD369
:103D1000FF2009F491C186ED94E060E035D421E004
:103D20002EAF8091AB03813009F48CC18091A30345
:103D3000882309F40CC1E090A703F8946E2C772433
:103D400076EC872E75E3972E860C971CD4018C9108
:103D500081FDF0C08C9182FDEDC08C9184608C93CC
:103D600081E07894882309F441C08091A3038823DB
:103D700009F054C12B966EAD7FAD2B978091A703B0
:103D8000A0900936B0900A36C0900B36D0900C3611
:103D9000A80EB11CC11CD11C27968CAD9DADAEAD3B
:103DA000BFAD2797A80EB91ECA1EDB1E80E090E0AB
:103DB0002091A60330E040E050E00E94893DA60E2D
:103DC000B71EC81ED91E0CD38091C335882309F4B1
:103DD00013C1C801B601A5012E2DE9DA05D3D4011E
:103DE0008C9182608C938C918B7F8C938091A703B4
:103DF000882301F5FF2059F085B1B8E08B2785B9FC
:103E00008091AB03823018F081508093AB032091F6
:103E1000AA03275E2093AA032D3708F008C130E0DB
:103E20008091A8039091A903821B930B9093890022
:103E3000809388008091A303882309F48FC052E304
:103E4000F52E05C08EE40E94FF10FA9431F08091A7
:103E50009F038823B9F34201BBCD80919F03882340
:103E6000D1F70E94FF10F394EF2DEC30B1F72FEF54
:103E70003FEF3093A5032093A4030E94DA100E9421
:103E8000DA100E94DA1080919F03882321F78EEFC9
:103E90000E94FF1080919F038823E9F622968FAD40
:103EA00022970E94FF1080919F038823A1F62E96EF
:103EB0008FAD2E970E94FF1080919F03882359F6A3
:103EC0008091A7038F5F0E94FF1080919F0388233A
:103ED00011F682E00E94FF10F090A4038091A503E8
:103EE00090919F03992309F0B6CF0E94FF10809113
:103EF0009F03882309F0AFCF8F2D0E94FF10FF246E
:103F000008C08EE40E94FF10F3943F2D363109F46F
:103F1000A8C180919F038823A1F39DCF80E464E032
:103F2000A6D28CED94E060E02FD380919F0388238C
:103F3000E1F359CE80E015CF8091A303882309F4E3
:103F400052CE80919D038C1509F039CE4CCEE09075
:103F5000A70323963FAD2397E30EEFCE27E3E22E90
:103F6000F12C0AC08FEF0E94CB100894E108F108F1
:103F7000E114F10409F489C080919F03882391F32F
:103F80006ACF22E146CE80919903815080939903B4
:103F9000C80161E00E94BB2E80919903882389F0BB
:103FA000FF249F2DADE09A9FB00111246D537E4CEC
:103FB000C80141E00E94D92EF39480919903F8162C
:103FC00080F310926B0310926A0389D3C8010E9498
:103FD0003506C8010E9448088FEF99E6A8E1815094
:103FE0009040A040E1F700C00000F2CCC80122964A
:103FF0006FAD229726DA86CE9301322F2227330F18
:104000002D533C4FC801B601A501EED4882309F019
:10401000E5CE89EF91E00E941716E0CE28969FAD7D
:10402000289729968FAD2997692F782FA7CE1092C0
:10403000AA0320E030E0F4CE80ED94E060E0A4D26A
:104040002B9A1EAE1092AB0380E065E010D28AEB93
:1040500094E060E099D26ACEF0909903AF2DBDE074
:10406000AB9FC00111248D539E4C6CE673E04DE074
:1040700050E00E94393EF394F0929903C8016CE637
:1040800073E041E00E94D92E9CCF8091A60382303C
:1040900009F4E4C082E0F82EE090A70380919F032A
:1040A000882309F0D8CE85ED0E94CB1080919F0324
:1040B000882309F0D0CE8AEA0E94CB1080919F031A
:1040C000882309F0C8CE86E90E94CB1080919F0317
:1040D000882309F0C0CE2C968FAD2C970E94CB1070
:1040E00080919F03882309F0B6CEE091A703F0E00A
:1040F000E458FE4F84910E94CB1080919F03882347
:1041000009F0A9CE2D968FAD2D970E94CB108091EE
:104110009F03882309F09FCEEF2DF0E0E458FE4F77
:1041200084910E94CB1080919F03882309F093CE45
:104130002196EFAD2197EE252FADE227EF25EF7306
:10414000F0E0E458FE4F84910E94CB1080919F03D1
:10415000882309F080CE8EED0E94CB1080919F03C2
:10416000882309F078CE8AEA0E94CB10BAE0FB2EB1
:1041700080919F03882309F06ECE8FEF0E94CB10B1
:10418000FA94B1F780919F03882309F064CE85EDFE
:104190000E94CB1080919F03882309F05CCE8AEAAD
:1041A0000E94CB1080919F03882309F054CE8DEAA2
:1041B0000E94CB1080919F03882309F04CCEE091A0
:1041C000A703F0E0E458FE4F84910E94CB10C30196
:1041D000982F8827990F8D539C4F0E94261180910C
:1041E0009F03882309F037CE8EED0E94CB1080917B
:1041F0009F03882309F02FCE8AEA0E94CB1080917A
:104200009F03882309F027CE8FEF0E94CB102296C0
:104210008FAD22976091A70395D88093A7034B9BFE
:104220006ACD2296DFAC229742014598429A1092BD
:10423000A103C8016D2D05D98FE79AE1A6E0815051
:104240009040A040E1F700C000000E94BF15C801E7
:104250000E943506C8010E944808BACB92E2F92EA6
:104260001BCF4CE0F42E80919F03882309F0F3CDFF
:104270000E94FF10FA94B9F78FEF9FEF9093A50378
:104280008093A4030E94DA100E94DA100E94DA10D0
:1042900080919F03882309F0DECD8BEF0E94FF10F1
:1042A0006301DC2CCC24DD0CA3ECB3E0CA0EDB1ED6
:1042B000EE24FF240BC00E94FF100894E11CF11CA7
:1042C000F0E0EF16F2E0FF0609F468C0F601819114
:1042D0006F0190919F03992371F3BDCD00D000D061
:1042E00000D0EDB7FEB731964DEA842E43E0942E10
:1042F000ADB7BEB712969C928E92119736E1E32E1F
:10430000F12CF382E28287EF92E0958384830E940E
:10431000483EF40101900020E9F73197E819F909C6
:104320002DB73EB72A5F3F4F0FB6F8943EBF0FBE82
:104330002DBF8E2F8195880F865D64E098D0C401D3
:1043400060E044E5A0D08DB79EB70A970FB6F89409
:104350009EBF0FBE8DBFEDB7FEB73196ADB7BEB7EE
:1043600012969C928E921197F382E28283E093E000
:10437000958384838981868317828B8180871186C8
:104380000E94483EEDB7FEB73A960FB6F894FEBFCE
:104390000FBEEDBF80E00E94240A09CBF090A40379
:1043A0008091A50390919F03992309F054CD0E9419
:1043B000FF1080919F03882309F04DCD8F2D0E941F
:1043C000FF1025CF81E090E00C94110A80E090E08E
:1043D0000C94110A14BC83E085BD81E085BB08956F
:1043E00081E080936E00089510926E0008951F92F0
:1043F0000F920FB60F9211248F939F93AF93BF9399
:104400008091113690911236A0911336B0911436E6
:104410000196A11DB11D8093113690931236A09381
:104420001336B0931436BF91AF919F918F910F9037
:104430000FBE0F901F9018952FB7F894609111360A
:104440007091123680911336909114362FBF0895D3
:1044500090E59CBD1DBC882341F05E9A2A986EBDF4
:104460000DB407FEFDCF2A9A08955E98F7CF1F93EB
:10447000162F682F606880E0EBDF612F606480E0BA
:10448000E7DF1F910895AF92BF92CF92DF92EF9234
:10449000FF920F931F93CF93DF93D62EC42EE82E57
:1044A000F92EBB248FE7A82EF70101917F0100238D
:1044B00059F4DF91CF911F910F91FF90EF90DF9012
:1044C000CF90BF90AF900895BC1498F70D3609F1C6
:1044D00083E0089F80011124E801C85FD84F065F80
:1044E000184FFE016491660FD1106A2581E0B0DF9C
:1044F000B394C017D10749F4BC14B0F6DD20C1F164
:104500006FE781E0A5DFB394CFCF2196BC1460F6AE
:10451000E8CFDD2079F163E481E09ADFB394BC1445
:1045200008F0C2CFDD2051F16BE781E091DFB39459
:10453000BC1408F0B9CFDD2029F167E681E088DFFF
:10454000B394BC1408F0B0CFDD20D1F06BE781E06C
:104550007FDFB394BC1408F0A7CFDD2069F067E4D7
:1045600081E076DFB394BC1408F09ECFDD2041F6E5
:1045700060E0C7CF6CE3D0CF68E3F2CF64E0D5CF83
:1045800064E0E5CF68E1DACFCF92DF92EF92FF925D
:104590000F931F93CF93DF93D62E8C010F5F1F4F86
:1045A0002FE7C22EF8013197E491EE2331F1ED3679
:1045B00079F183E0E89FF0011124EF01C85FD84F43
:1045C0009BE0E92E97E0F92EEE0EFF1EFE016491AE
:1045D000660FD1106C2581E03BDF2196CE15DF05FB
:1045E000A9F7DD2099F06FE781E032DF0F5F1F4F01
:1045F000F8013197E491EE23D1F6DF91CF911F912D
:104600000F91FF90EF90DF90CF90089560E0ECCF96
:10461000DD2089F081E063E41BDF81E06BE718DFD8
:1046200081E067E615DF81E06BE712DF81E067E498
:104630000FDF6FE7D9CF81E06CE30ADF81E064E050
:1046400007DF81E068E104DF81E064E001DF81E011
:1046500068E3FEDE60E0C8CFEF92FF920F931F93F6
:10466000CF93DF93E82EF92EF70101917F0100230C
:10467000E1F00D3609F183E0089F80011124E80183
:10468000C85FD84F055F184FFE016491606481E0F8
:10469000DFDE2196C017D107B9F781E060E4D8DEEC
:1046A000F70101917F01002321F7DF91CF911F9145
:1046B0000F91FF90EF90089581E06EE5C9DE81E0F3
:1046C00062E4C6DE81E06CE4C3DE81E062E4C0DE69
:1046D00081E06CE5BDDE81E060E4BADEC5CFCF935A
:1046E000DF93C8EFD1E081E060E0B2DE2197D9F737
:1046F000DF91CF91089584EB8093153684E1809308
:10470000163684E080931736569A279A259A229A6D
:10471000209A2A9880E090E00E948840813FE1F052
:1047200080E090E061EF0E9490406091153681E05A
:1047300090E00E94904080E061E28ADE6091153650
:1047400080E086DE6091163680E082DE80E060E206
:104750007FDE80E06CE07CCE81E090E00E948840CB
:1047600080931536E8CFFC014181842F90E09C01B5
:104770003595279520652CBD40FD06C081E046306B
:1047800019F08DBD2C98089580E08DBD2C9808956A
:10479000BF92CF92DF92EF92FF920F931F93CF932E
:1047A000DF938C016B017A0147DEEB01BB24BA94E5
:1047B000BEBC0DB407FEFDCF8EB5F80182838F3FDE
:1047C000B1F43ADE6C1B7D0B81E06D32780780F32B
:1047D00081E1F80180832C9A80E0DF91CF911F91D5
:1047E0000F91FF90EF90DF90CF90BF9008958E3F94
:1047F00019F08FE08083EFCFE114F104F1F0089419
:10480000E108F1088FEF8EBDE114F10471F0F601BB
:1048100080E090E03FEF0DB407FEFDCF2EB5219371
:104820003EBD01968E159F05B0F30DB407FEFDCF7A
:104830008EB5F601EE0DFF1D80838FEF8EBD0DB49A
:1048400007FEFDCF8EB58FEF8EBD0DB407FEFDCFF9
:104850008EB52C9A81E0C1CF0F931F93CF93DF9336
:10486000EC018B0180DFCE01B80140E052E090DF27
:10487000DF91CF911F910F910895FF920F931F9396
:10488000CF93DF93EB01D8DD8B01FF24FA94FEBCBC
:104890000DB407FEFDCF8EB58F3F69F0CDDD601BF7
:1048A000710B6C177D0798F380E0DF91CF911F911A
:1048B0000F91FF90089581E0DF91CF911F910F91AB
:1048C000FF900895DF92EF92FF920F931F93CF9383
:1048D000DF93EC01D62E79018A0145DFCE016CE22F
:1048E00071E0CBDF8D2D80648EBD0DB407FEFDCF52
:1048F00028E130E0D801C701022E04C0B695A79583
:10490000979587950A94D2F78EBD0DB407FEFDCF1B
:10491000285030408FEF283F380761F7DD20E9F05D
:104920008D2D883001F587E88EBD0DB407FEFDCFD3
:104930008D2D8C30D1F02FEF9FEF9EBD0DB407FE73
:10494000FDCF8EB58A8387FD0AC0DF91CF911F917D
:104950000F91FF90EF90DF90089585E9E5CF222336
:10496000A1F32150EACF8FEFDFCF8FEF8EBD0DB4D3
:1049700007FEFDCF8EB5DFCFCF93DF93EC01F3DEE3
:10498000CE016CE020E030E0A9019CDF882339F003
:1049900083E088832C9A80E0DF91CF9108952C9A50
:1049A00081E0DF91CF910895CF93DF93EC019A01DD
:1049B000AB018B81833039F069E0220F331F441F34
:1049C000551F6A95D1F7CE0162E17CDF882339F06B
:1049D00085E088832C9A80E0DF91CF9108952C9A0E
:1049E00081E0DF91CF910895CF92DF92EF92FF9215
:1049F0000F931F93CF93DF93EC017A018B01690131
:104A00008B81833039F0A9E0EE0CFF1C001F111FD1
:104A1000AA95D1F7CE0161E1A801970153DF882360
:104A200069F084E088832C9A80E0DF91CF911F9118
:104A30000F91FF90EF90DF90CF900895CE01B601D7
:104A400040E052E0A5DEF1CF8F929F92BF92CF92CD
:104A5000DF92EF92FF920F931F93DF93CF930F920A
:104A6000CDB7DEB74C01B62EFC0113821082E4DC18
:104A70008B01249A2C9A2698259A279A249A2C9A64
:104A800085E0F401818382E58CBD1DBC8AE09FEF47
:104A90009EBD0DB407FEFDCF8150D1F7C40160E08B
:104AA00020E030E0A9010EDF782FF401828381300D
:104AB000C9F0C2DC601B710BF7E0613D7F0770F34A
:104AC00081E0F40180832C9A80E00F90CF91DF91F8
:104AD0001F910F91FF90EF90DF90CF90BF909F902C
:104AE0008F900895C40168E02AEA31E040E050E088
:104AF0007983E8DE798182FF1FC0F4017383CC24BF
:104B0000DD247601C40167E320E030E0A901DADEAC
:104B1000C40169E2A7019601D5DEF40182838823EE
:104B2000D9F08ADC601B710BF7E0613D7F0750F321
:104B30008AE0F4018083C7CF84E02FEF2EBD0DB44F
:104B400007FEFDCF9EB5F40192838150B9F79A3AE2
:104B500079F082E08083B7CF83818230B1F02C9AE4
:104B6000FB2DF73070F088E1F401808380E0ADCF59
:104B700082E0F4018383C12CD12CE12CB0E4FB2E24
:104B8000C1CFF401B18281E0A0CFC4016AE320E08B
:104B900030E0A90197DE882321F088E0F4018083CA
:104BA00092CF8FEF8EBD0DB407FEFDCF8EB5807C0A
:104BB000803C19F483E0F401838383E09FEF9EBD82
:104BC0000DB407FEFDCF2EB58150C9F7C8CFFC014B
:104BD0006EBDA42FB52F80E090E00DB407FEFDCF91
:104BE0002C912EBD0DB407FEFDCF11962C9111977F
:104BF0002EBD0296129622E08030920771F70DB416
:104C000007FEFDCF8FEF8EBD0DB407FEFDCF8FEFFA
:104C10008EBD0DB407FEFDCF8FEF8EBD0DB407FE28
:104C2000FDCF8EB582838F71853029F083E180833B
:104C30002C9A80E0089581E008950F931F93CF93FD
:104C4000DF93EC018B018FDDCE0168E572E015DEAC
:104C5000882349F485E188832C9A80E0DF91CF9105
:104C60001F910F910895CE016CEFA801B0DF88234A
:104C700089F32C9A81E0DF91CF911F910F910895D4
:104C8000CF92DF92EF92FF920F931F93CF93DF9318
:104C9000EC017A018B0169018B81833039F089E065
:104CA000EE0CFF1C001F111F8A95D1F7CE0168E1A1
:104CB000A801970107DE882369F086E088832C9A93
:104CC00080E0DF91CF911F910F91FF90EF90DF90E7
:104CD000CF900895CE016EEFA60179DF882379F396
:104CE000CE0168E572E0C9DD882319F487E1888385
:104CF000E6CFCE016DE020E030E0A901E3DD8823BE
:104D000019F086E18883DBCF8FEF8EBD0DB407FEEF
:104D1000FDCF8EB58823A9F72C9A81E0D2CFAF9230
:104D2000BF92CF92DF92EF92FF920F931F93CF9398
:104D3000DF93EC015A016B017801890167E320E000
:104D400030E0A901BFDDCE0167E1A8019701BADD1E
:104D5000882379F089E088832C9A80E0DF91CF91D5
:104D60001F910F91FF90EF90DF90CF90BF90AF9089
:104D700008958B81833039F099E0AA0CBB1CCC1CC0
:104D8000DD1C9A95D1F7CE0169E1A60195019ADD66
:104D9000882319F087E08883DFCF2C9A81E0DECF6B
:104DA000CF93DF93EC01DFDCCE0168E572E065DDD7
:104DB000882359F08DEF8EBD0DB407FEFDCFCE01D7
:104DC00068E572E05ADD882339F482E188832C9A01
:104DD00080E0DF91CF9108952C9A81E0DF91CF910F
:104DE0000895CF93DF93EC019C012C5F3F4F898D99
:104DF0009A8D41E050E060E070E00E9483318823AA
:104E0000D9F08D899E89AF89B88D0097A105B1052C
:104E100079F48C819D81AE81BF818D8B9E8BAF8B10
:104E2000B88F89818068898381E0DF91CF9108956F
:104E300081E0DF91CF91089580E0DF91CF910895D7
:104E4000CF92DF92EF92FF921F93CF93DF93EC010B
:104E500089899A89AB89BC89803E2FEF92072FE11F
:104E6000A20720E0B20748F080E0DF91CF911F91C8
:104E7000FF90EF90DF90CF900895CE01B2DF8823AE
:104E800099F30E94572F882379F3E98DFA8DCC800E
:104E9000DD80EE80FF808EEF9FEFAFEFBFEFC80E9B
:104EA000D91EEA1EFB1E058404C0CC0CDD1CEE1CC2
:104EB000FF1C0A94D2F786859785A089B189C80E10
:104EC000D91EEA1EFB1E81E080932438C0921E3654
:104ED000D0921F36E0922036F092213680E092E0A8
:104EE000E2E2F6E3DF019C011D9221503040E1F740
:104EF000E98DFA8D84818230C0F011E006C01F5F19
:104F0000E98DFA8D8481181780F4B701A601410F4D
:104F1000511D611D711D809122389091233822E22C
:104F200036E3AEDE882359F79FCF20E032E040E041
:104F300050E0058404C0220F331F441F551F0A94FC
:104F4000D2F789899A89AB89BC89820F931FA41FE4
:104F5000B51F898B9A8BAB8BBC8B81E086CFCF93AF
:104F6000DF93EC018C859D85AE85BF8541E066238E
:104F700009F440E0BC01CD01DAD7882381F028890B
:104F800030E0220F331F22953295307F3227207F69
:104F900032272E5D394CC901DF91CF91089520E071
:104FA00030E0C901DF91CF9108956F927F928F9287
:104FB0009F92AF92BF92CF92DF92EF92FF920F93A8
:104FC0001F93DF93CF9300D000D0CDB7DEB76C0135
:104FD0004B013A01DC015596ED90FD900D911C912D
:104FE0005897E114F10401051105F1F05E010894F0
:104FF000A11CB11C10C0D801C7010196A11DB11D93
:1050000029813A814B815C8182179307A407B507F8
:10501000F9F47C018D01F601818D928DB801A70113
:105020009501CAD7882339F780E00F900F900F9031
:105030000F90CF91DF911F910F91FF90EF90DF9034
:10504000CF90BF90AF909F908F907F906F9008957A
:10505000D60159966D917C915A97FB0187898031D1
:1050600009F44CC0283F8FEF38078FEF48078FE0D7
:105070005807D0F2F60185899689A789B08D0297E5
:10508000A109B109FB01058404C0880F991FAA1F5B
:10509000BB1F0A94D2F72685378540895189820F34
:1050A000931FA41FB51FF40180839183A283B38350
:1050B000FB0186859785A089B1890197A109B1096E
:1050C0002481820F911DA11DB11DA80197012250BD
:1050D000304040405040058404C0220F331F441F1D
:1050E000551F0A94D2F7820F931FA41FB51FF30117
:1050F00080839183A283B38381E097CF283FFFEF22
:105100003F07F0E04F07F0E05F0708F0B3CF8CCF28
:10511000E82FF92F80E090E03EE209C0DB01A90F03
:10512000B11D2C939F5F8F5F31968B3061F0208192
:105130002032C9F3883091F7DB01A90FB11D3C93F0
:105140009F5F2081EBCF690F711DFB0110820895D5
:105150001F93FB012BE030E231932150E9F7A82F98
:10516000B92F30E017E09A2F8B2F2D91222351F485
:10517000FA019083818381E0FB019081903279F084
:105180001F9108952F32A1F32E3261F085E898E047
:10519000FC010196E491EE2351F02E17C9F780E04F
:1051A0001F9108951A30D9F338E01AE0DCCF1317B5
:1051B000B0F32132A0F32F3790F7FB01E30FF11D7D
:1051C000822F81568A3108F4205220833F5FCBCF53
:1051D0000F931F93CF93DF93EC018B018B81882377
:1051E00031F4FB018789803141F08032F1F180E0B8
:1051F000DF91CF911F910F91089582E08B831D8ADB
:105200001E8A1F8A188E808D918DA0E0B0E0880FD5
:10521000991FAA1FBB1F880F991FAA1FBB1F880FAA
:10522000991FAA1FBB1F880F991FAA1FBB1F880F9A
:10523000991FAA1FBB1F898B9A8BAB8BBC8B1A8FB4
:10524000098F81E089831C821D821E821F8218863D
:1052500019861A861B861C861D861E861F86188A3E
:10526000DF91CF911F910F91089583E08B83F80117
:10527000428D538D648D758D4D8B5E8B6F8B788FCA
:105280009E012F5E3F4FC80124D78823C1F6AFCFC0
:105290002F923F924F925F926F927F928F929F9246
:1052A000AF92BF92CF92DF92EF92FF920F931F9334
:1052B000CF93DF938C01362FE72F2A01DC01139661
:1052C0002C911397222329F011968C91119780FD30
:1052D00016C02FEF3FEFC901DF91CF911F910F91C2
:1052E000FF90EF90DF90CF90BF90AF909F908F9006
:1052F0007F906F905F904F903F902F900895E801BE
:10530000C988DA88EB88FC88488559856A857B8559
:105310004201AA24BB24D701C601841B950BA60B0E
:10532000B70B88169906AA06BB0608F093C041146D
:10533000510409F4BEC0832E9E2E6201A4E02A2EE1
:10534000312C200E311E612CF2E07F2E60C0FF2038
:1053500009F07AC0411551056105710509F0ABC02E
:10536000E8018D899E89AF89B88D8C839D83AE833A
:10537000BF8346855785608971894F0D511D611D19
:10538000711D0297A109B109058404C0880F991FF6
:10539000AA1FBB1F0A94D2F7480F591F6A1F7B1F11
:1053A000E301CA19DB09CC16DD0608F4E601E2E0E8
:1053B000C030DE0709F452C0CB01BA0140E0B7D5D6
:1053C000882309F486CF95012E5D394CC401B901BB
:1053D000AE010E94223EAE0160E070E0F8018085DF
:1053E0009185A285B385480F591F6A1F7B1FD8017D
:1053F00018964D935D936D937C931B97CC1ADD0AA1
:1054000009F457C08C0E9D1E13962C911397EFEF45
:10541000AE2EE1E0BE2EA422B5222230B9F1D80191
:105420005996ED91FC915A97DB01CA0129E0B69596
:10543000A795979587952A95D1F7F480FA94F82245
:10544000A114B10409F483CFE8018C819D81AE8160
:10545000BF818FCF2601441A550A69CF80911E362D
:1054600090911F36A0912036B091213648175907E8
:105470006A077B0709F4A0CF8091223890912338E6
:105480009401B2DA882309F0A6CF23CF39E07695CC
:105490006795579547953A95D1F7E801E98DFA8DCB
:1054A000828D938DA48DB58D480F591F6A1F7B1F68
:1054B00077CF920110CFD80114964D915D916D91E7
:1054C0007C911797CF01910177D5882309F401CFFB
:1054D000E801E98DFA8D8C819D81AE81BF8149CF34
:1054E000DF93CF930F92CDB7DEB7BE016F5F7F4FD3
:1054F00041E050E0CDDE8130910539F02FEF3FEFF4
:10550000C9010F90CF91DF910895298130E0C90141
:105510000F90CF91DF910895EF92FF920F931F9319
:10552000CF93DF93EC018B81823050F420E030E0A8
:10553000C901DF91CF911F910F91FF90EF900895D6
:10554000E884F9840A851B85CE01CADF97FDEECF7A
:1055500088859985AA85BB854F96A11DB11D888731
:105560009987AA87BB87D801C70115E0B695A7958B
:10557000979587951A95D1F78F70282F30E0220FD5
:10558000331F22953295307F3227207F32272E5DC0
:10559000394CCECF8F929F92AF92BF92CF92DF9233
:1055A000EF92FF920F931F93CF93DF93EC014A0189
:1055B0005B012B81222309F465C089899A89AB8913
:1055C000BC8984179507A607B70708F45BC022308B
:1055D00009F452C081149104A104B10409F46AC011
:1055E000488559856A857B85E98DFA8D258530E06A
:1055F000275F3F4FDB01CA010197A109B109022EC4
:1056000004C0B695A795979587950A94D2F785011A
:1056100074010894E108F1080109110904C0169504
:105620000795F794E7942A95D2F7E816F9060A0742
:105630001B07B0F58D899E89AF89B88D8C839D83BA
:10564000AE83BF8384E0C82ED12CCC0EDD1E0FC0EC
:105650004C815D816E817F81898D9A8D9601ACD45C
:105660000894E108F10801091109882359F0E114AF
:10567000F1040105110561F788869986AA86BB8623
:1056800081E001C080E0DF91CF911F910F91FF90E9
:10569000EF90DF90CF90BF90AF909F908F90089544
:1056A000411551056105710529F2E81AF90A0A0B3D
:1056B0001B0BC8CF1C821D821E821F821886198672
:1056C0001A861B8681E0DFCF0F931F93CF93DF9362
:1056D000EC018B81882349F0898187FD0EC0E7D3D7
:1056E000DF91CF911F910F91089581E0888380E031
:1056F000DF91CF911F910F910895CE0161E02FDCD2
:105700008C01009791F3FC018081853E71F38B81C0
:105710008230F8F08D899E89AF89B88DF801938F1A
:10572000828FB58BA48BE0911A36F0911B3630979F
:1057300059F0B8016A5E7F4FC80148960995F80193
:10574000808D918D938B828B89818F778983AFD365
:10575000C7CF89899A89AB89BC89848F958FA68F99
:10576000B78FD8CFCF93DF93EC01AEDF1B82DF91F1
:10577000CF9108956F927F928F929F92AF92BF9236
:10578000CF92DF92EF92FF920F931F93DF93CF930D
:1057900000D000D0CDB7DEB77C015A016B01DC012F
:1057A00013968C9113978130A1F080E00F900F90A9
:1057B0000F900F90CF91DF911F910F91FF90EF907D
:1057C000DF90CF90BF90AF909F908F907F906F9021
:1057D000089511968C91119781FFE7CFF701818988
:1057E0009289A389B48984179507A607B707E8F2B9
:1057F0000097A105B10529F1F701608471848284C5
:105800009384C701B601A501C5DE882371F2A114F6
:10581000B104C104D104B9F4D70155964D915D91FD
:105820006D917C91589759968D919C915A97A3D6DA
:10583000882309F4BACFF701158A168A178A108EC1
:1058400040C081E0B3CFD70114964D915D916D9129
:105850007C91179759968D919C915A979E012F5F35
:105860003F4FAAD3882309F4A0CFD7015996ED91D1
:10587000FC915A9749815A816B817C81878980315B
:10588000C9F1483F8FEF58078FEF68078FE078071F
:10589000C0F4CF0170D6882309F487CFD7011496BE
:1058A0004D915D916D917C91179759968D919C9139
:1058B0005A970FEF1FEF2FEF3FE086D4882309F4AC
:1058C00074CFF701A18AB28AC38AD48A81818068A1
:1058D0008183C701F9DE882309F467CFB601A501EA
:1058E0006A147B048C049D0410F4B401A301C70165
:1058F00051DE5CCF483FBFEF5B07B0E06B07B0E025
:105900007B07F8F6C6CF1F93CF93DF93EC01142FDC
:10591000E62FF0E0EE0FFF1FE295F295F07FFE27F5
:10592000E07FFE27DF01AE5DB94C1B968C911B9783
:10593000817149F0842F827131F01B8280E0DF9108
:10594000CF911F91089580911E3690911F36A0919E
:105950002036B09121368C879D87AE87BF87688BB4
:10596000EE5DF94C84899589A0E0B0E0DC019927CF
:1059700088278D8B9E8BAF8BB88F428D538D60E0C7
:1059800070E0482B592B6A2B7B2B4D8B5E8B6F8BDA
:10599000788F838590E0887190700097F1F4848D02
:1059A000958DA68DB78D898B9A8BAB8BBC8B81E047
:1059B0008B83812F8F7089831C821D821E821F82A0
:1059C000188619861A861B8614FD17C015FD1EC081
:1059D00081E0DF91CF911F9108958031910509F009
:1059E000ACCF9E012F5E3F4F898D9A8D72D3882355
:1059F00009F4A3CF84E08B83DCCFCE0140E050E0FC
:105A0000BA01B8DE882311F780E099CF49895A8915
:105A10006B897C89CE01BEDD92CF8F929F92AF922F
:105A2000BF92CF92DF92EF92FF920F931F93CF938B
:105A3000DF935C01EB01C42E952E822E898D9A8D09
:105A4000D5015A969C938E935997CB0140E050E034
:105A5000BA01A0DDDD24E884F9840A851B858989E3
:105A60009A89AB89BC89E816F9060A071B0708F072
:105A700040C0CE0151DDFC01009709F476C0D80189
:105A8000C70115E0B695A795979587951A95D1F713
:105A9000182F1F708081882391F0853E81F08C2D16
:105AA000992DBF014BE050E00E94153E009799F6FA
:105AB00087FC5BC0C501612F482D25DF57C0DD2065
:105AC000A9F420911E3630911F3640912036509116
:105AD0002136D5011C962D933D934D935C931F97D2
:105AE00050961C9350978081DD24D394882309F02D
:105AF000B2CF86FE3AC081FE38C0DD2009F043C037
:105B00008B81823091F1CE019BD9882371F1C2E261
:105B1000D6E310E07E01EC2FFF2D80E2DF011D9225
:105B20008A95E9F7DE018C2D992DFC018BE001901F
:105B30000D928150E1F7E0911A36F0911B363097C3
:105B400061F1BE01625F7F4FCE0140960995888961
:105B500099892E853F859B8B8A8B998F888F3F8B68
:105B60002E8BA5D1882309F0A5CF80E0DF91CF91BE
:105B70001F910F91FF90EF90DF90CF90BF90AF906B
:105B80009F908F900895F5011089C50161E0E7D9D4
:105B9000EC01009709F0BECFE8CF81E298E2998B43
:105BA000888B80E098E09F878E8720E038E081E254
:105BB00098E2D1CF2F923F924F925F926F927F9255
:105BC0008F929F92AF92BF92CF92DF92EF92FF920D
:105BD0000F931F93DF93CF93CDB7DEB7C454D0405C
:105BE0000FB6F894DEBF0FBECDBF2C013B018E0176
:105BF0000E5B1F4FD80111965C934E9325962FAFE5
:105C000025971C861F861FA21AA66115710509F427
:105C10005FC0FC018381882309F05AC0CA01DA0100
:105C20002C912F3209F470C073013CE0832E912C2B
:105C30008C0E9D1E64015E010894A11CB11C27E21C
:105C4000222E312C2C0E3D1EB501A80181DA8823AD
:105C500069F1D801ED91FC91119780818F3241F467
:105C60003196D8011196FC93EE9381918F32C9F34E
:105C7000882309F46FC0C601B701A50121E0CDDE7C
:105C80008823A1F0E614F70421F0C7011DDDF70118
:105C90001382C814D904C9F076016401D8018D912A
:105CA0009C91B501A80154DA882399F600E08AA5F1
:105CB000882321F0CE01879607DD1AA68F858823D9
:105CC00041F0CE010C9600DD04C061017401E6CF05
:105CD00000E0802FCC5BDF4F0FB6F894DEBF0FBE25
:105CE000CDBFCF91DF911F910F91FF90EF90DF908B
:105CF000CF90BF90AF909F908F907F906F905F906C
:105D00004F903F902F9008959A012F5F3F4FC90108
:105D1000F80131832083D9014C912F5F3F4F4F32DF
:105D2000B1F3F30123812250223008F47DCF87E2C2
:105D3000E82EF12CEC0EFD1ED30159966D917C914D
:105D40005A97C70145DA882309F4B0CFF80180815A
:105D500091816BCFC201B701A50125962FAD259783
:105D60005CDE082FA4CFFB01242F609118367091C0
:105D70001936AF011FCF0F931F93CF93DF93EC0121
:105D8000662399F08C010E5D1F4F10931936009316
:105D90001836C801E7DCBE016C5F7F4FC80118DA16
:105DA000DF91CF911F910F9108958C010E5D1F4FD0
:105DB000F0CFDF92EF92FF920F931F93DF93CF9379
:105DC000CDB7DEB76C970FB6F894DEBF0FBECDBF70
:105DD000FB01D42E19821C8220812F3229F122E26C
:105DE000E22EF12CE80EF91E8E010F5F1F4FC80145
:105DF000B701AF0121E0DEDE8823F1F08C81823033
:105E000070F1D701F8018BE101900D928150E1F71B
:105E1000DD2021F0F0921936E092183621E0C80119
:105E20002C8FA0DC2C8D0CC021812223C1F6642F85
:105E3000A2DF282F8C8102C08C8120E0882389F486
:105E4000822F6C960FB6F894DEBF0FBECDBFCF91F8
:105E5000DF911F910F91FF90EF90DF90089520E068
:105E6000EDCF8E010F5F1F4FDACF0F931F93CF93AC
:105E7000DF938C010E942425882331F480E0DF9198
:105E8000CF911F910F910895E8012496CE01B8019A
:105E900041E0CDD3882321F0C80161E06CDFEFCF72
:105EA000CE01B80140E0C3D3882341F3F5CF809100
:105EB0002438882311F481E0089540911E365091D2
:105EC0001F36609120367091213680912238909152
:105ED000233822E236E30E944026882321F14091B4
:105EE000253850912638609127387091283841150F
:105EF00051056105710521F41092243881E008955F
:105F0000809122389091233822E236E30E94402685
:105F1000882359F01092253810922638109227388D
:105F200010922838E9CF80E0089580E00895DF924C
:105F3000EF92FF920F931F937B018C01D42E8091DF
:105F40001E3690911F36A0912036B09121368E15C5
:105F50009F05A007B107F1F0AADF882339F480E09C
:105F60001F910F91FF90EF90DF900895809122385C
:105F700090912338B801A70122E236E30E94F4246D
:105F8000882369F3E0921E36F0921F360093203684
:105F900010932136DD2049F081E0809324381F9151
:105FA0000F91FF90EF90DF90089581E01F910F9186
:105FB000FF90EF90DF900895CF92DF92EF92FF92E3
:105FC0000F931F93CF93DF93EC017A018B0169014B
:105FD00089859A85AB85BC850196A11DB11D841765
:105FE0009507A607B70730F0EF89E03169F0E03296
:105FF00009F445C080E0DF91CF911F910F91FF9090
:10600000EF90DF90CF9008959927872F762F652FF7
:106010002B893C894D895E89620F731F841F951FF0
:1060200020911E3630911F364091203650912136F6
:10603000621773078407950729F040E078DF88230B
:10604000C9F2EF89E03169F18FE790E0A0E0B0E0BC
:10605000E822F9220A231B23F701EE0FFF1FEE0FA0
:10606000FF1FEE5DF94C80819181A281B381BF70E9
:10607000F60180839183A283B38381E0BCCFCB01FF
:10608000BA0127E096958795779567952A95D1F778
:106090002B893C894D895E89620F731F841F951F70
:1060A000BFCF8FEF90E0A0E0B0E0E822F9220A2312
:1060B0001B23F701EE0FFF1FEE5DF94C80819181EC
:1060C000A0E0B0E0F60180839183A283B38381E0F6
:1060D00092CF4F925F926F927F928F929F92AF92E8
:1060E000BF92CF92DF92EF92FF920F931F93DF93B5
:1060F000CF9300D000D0CDB7DEB78C0149835A834F
:106100006B837C832901842F952FA62FB72FAC0199
:10611000BD01CC24DD2476015E010894A11CB11CD4
:10612000612CE2E07E2E812C912CC801950144DF88
:10613000882309F447C0D401C301F801058404C0D1
:10614000880F991FAA1FBB1F0A94D2F7C80ED91E29
:10615000EA1EFB1E49815A816B817C8187898031CF
:1061600019F1483F8FEF58078FEF68078FE07807E6
:10617000E0F2F201C082D182E282F38281E00F90EC
:106180000F900F900F90CF91DF911F910F91FF9083
:10619000EF90DF90CF90BF90AF909F908F907F90C7
:1061A0006F905F904F900895483FFFEF5F07F0E0DA
:1061B0006F07F0E07F07E8F6C8019501FDDE882350
:1061C00009F0B9CF80E0DBCF4F925F926F927F9260
:1061D0008F929F92AF92BF92CF92DF92EF92FF92F7
:1061E0000F931F93CF93DF93EC016A017B0128018A
:1061F0003901423051056105710590F089859A8514
:10620000AB85BC850196A11DB11D84179507A60716
:10621000B70730F08F89803109F456C0803291F091
:1062200080E0DF91CF911F910F91FF90EF90DF9071
:10623000CF90BF90AF909F908F907F906F905F9026
:106240004F9008954A015B0117E0B694A794979484
:1062500087941A95D1F78B899C89AD89BE89880E60
:10626000991EAA1EBB1EC501B40141E060DE882351
:10627000B9F28F898031A9F18FE790E0A0E0B0E01A
:10628000C822D922EA22FB22F601EE0FFF1FEE0FF1
:10629000FF1FEE5DF94C40825182628273828A89CF
:1062A000823078F18D819E81AF81B885880D991DEE
:1062B000AA1DBB1D8093253890932638A0932738BC
:1062C000B093283881E0ADCF852E962EA72EBB2423
:1062D0008B899C89AD89BE89880E991EAA1EBB1E1A
:1062E000C2CF8FEF90E0A0E0B0E0C822D922EA222E
:1062F000FB22F601EE0FFF1FEE5DF94C518240824A
:10630000CECF81E08ECF2F923F924F925F926F92CD
:106310007F928F929F92AF92BF92CF92DF92EF9235
:10632000FF920F931F93DF93CF93CDB7DEB767979D
:106330000FB6F894DEBF0FBECDBF1C0149875A8748
:106340006B877C873E872D87FC0181859285A3859D
:10635000B4859C01AD012F5F3F4F4F4F5F4F2D83A1
:106360003E834F835887ED85FE8540805180628053
:106370007380411451046104710409F4BEC008948F
:10638000411C511C611C711C1F860097A105B105A1
:1063900009F454C0D301C201CC24DD2476018E015E
:1063A0000F5F1F4F4C8A5D8A6E8A7F8A2EC04C0118
:1063B0005D01C101B501A4019801FEDD882309F446
:1063C0003DC089819A81AB81BC810097A105B1054F
:1063D00009F44EC0A50194012F5F3F4F4F4F5F4F0F
:1063E0002C8B3D8B4E8B5F8BDA01C9010894C11C4D
:1063F000D11CE11CF11CF1012185328543855485B6
:10640000C216D306E406F506C8F44D805E806F80A0
:106410007884481659066A067B0648F682E0882E7C
:10642000912CA12CB12C8C8A9D8AAE8ABF8AC10185
:10643000B501A4019801C0DD882319F680E06796B4
:106440000FB6F894DEBF0FBECDBFCF91DF911F9185
:106450000F91FF90EF90DF90CF90BF90AF909F9003
:106460008F907F906F905F904F903F902F90089506
:10647000D501C4010196A11DB11D2C013D012C893E
:106480003D894E895F89421A530A640A750A298533
:106490003A854B855C85421653066406750609F0FD
:1064A000A5CF4C885D886E887F88C101B501A401A5
:1064B0000FEF1FEF2FEF3FE087DE882309F4BECFF9
:1064C000481459046A047B0458F59501840107C0F7
:1064D000970186014C145D046E047F0408F5680181
:1064E00079010894C108D108E108F108C101B70198
:1064F000A6016ADE882361F7A1CFF10140805180B7
:1065000062807380F1E0FF8729853A854B855C8541
:10651000213031054105510509F437CF1F8635CFAC
:10652000AD85BE854D915D916D917C91139741151F
:10653000510561057105C1F4ED85FE8540825182EA
:1065400062827382FF85FF2369F00894411C511C0D
:10655000611C711CD1014D925D926D927C921397DA
:1065600081E06DCF81E06BCFC101930182012CDE10
:10657000882311F763CFAF92BF92CF92DF92EF9251
:10658000FF920F931F93DF93CF9300D000D0CDB72E
:10659000DEB76C017A018B0182E090E0A0E0B0E010
:1065A000F60180839183A283B3835E010894A11CCA
:1065B000B11CC601B801A7019501FEDC882339F1A1
:1065C000C601B801A70100E010E09801FDDD8823B5
:1065D000F1F0E980FA800B811C81F6018789803116
:1065E00059F088EFE8168FEFF8068FEF08078FE075
:1065F0001807F8F281E00CC0F8EFEF16FFEFFF0686
:10660000F0E00F07F0E01F07A0F281E001C080E09A
:106610000F900F900F900F90CF91DF911F910F91DE
:10662000FF90EF90DF90CF90BF90AF9008956F9262
:106630007F928F929F92AF92BF92DF92EF92FF92E2
:106640000F931F93CF93DF93EC01142F7093233894
:10665000609322381F8A82E090E0A0E0B0E0888357
:106660009983AA83BB831092243810922538109204
:10667000263810922738109228388FEF9FEFDC01D0
:1066800080931E3690931F36A0932036B093213608
:10669000442309F444C0453078F080E0DF91CF9185
:1066A0001F910F91FF90EF90DF90BF90AF909F9060
:1066B0008F907F906F90089560E070E0CB0140E094
:1066C00036DC882351F3212F30E022953295307F3C
:1066D0003227207F32272E5E394CF901E254FE4FDB
:1066E000808190E08F7790700097B9F6F901E653BA
:1066F000FE4F80819181A281B38184369105A105ED
:10670000B10558F22A533E4FF901E080F180028131
:106710001381E114F1040105110521F4BECFEE242B
:10672000FF248701C801B70140E001DC882309F498
:10673000B4CF80912D3690912E36F2E080309F07B5
:1067400009F0ABCF20913236222309F4A6CF8091F5
:10675000303690913136009709F49FCF60912F36F3
:10676000662309F49ACF2A8B6C831D8670E080E043
:1067700090E041E050E008C0282F2F5F2D87019660
:106780008930910509F489CFD82E9A01082E02C0CC
:10679000220F331F0A94E2F72617370769F7609133
:1067A0003836709139366115710509F47FC080E083
:1067B00090E06D837E838F839887809030369090B1
:1067C0003136AA24BB248E0C9F1CA01EB11E8B8ABE
:1067D0009C8AAD8ABE8A6090333670903436798E4A
:1067E000688E2091323630E040E050E00E94893DD2
:1067F000680D791D8A1D9B1D6A8F7B8F8C8F9D8FE5
:106800009301220F331F22953295307F3227207F4C
:10681000322721503E4F232F3327269540E050E06A
:10682000260F371F481F591F2E873F87488B598BCC
:106830008091353690913636009709F440C0A0E03B
:10684000B0E0E21AF30A040B150BE80EF91E0A1F5A
:106850001B1F04C016950795F794E794DA94D2F7B6
:10686000E986FA860B871C8725EFE2162FE0F206F1
:1068700020E0020720E0120758F185EFE8168FEFBD
:10688000F80680E0080780E0180730F180914E3666
:1068900090914F36A0915036B09151368A8F9B8F90
:1068A000AC8FBD8F80E28F8B81E0F8CE6091463651
:1068B0007091473680914836909149367ACF8091D1
:1068C000423690914336A0914436B0914536B9CFC7
:1068D0008CE08F8B80E0E2CE80E18F8B81E0DECE9A
:1068E000CF93DF93DC01CD91DC9111971C161D062F
:1068F000DCF41296E0E0F0E020E030E0A901542F53
:10690000432F322F22276D9170E080E090E0262BFC
:10691000372B482B592B3196EC17FD0781F7B9011E
:10692000CA01DF91CF91089520E030E0A901F7CFAF
:10693000CF93DF93FB01DC012D913C91B9016E5F98
:106940007F4FEC01C60FD71FE60FF71FD901119635
:10695000A40FB51F2115310599F0215030408A91BF
:1069600092914115510519F06C9186239623119748
:10697000891781F320E030E0C901DF91CF910895BC
:1069800021E030E0C901DF91CF910895CF93DF93EB
:10699000FB0120813181DC012D933C93A081B181E9
:1069A000109701F1BD01615070401296EA0FFB1F74
:1069B000EA01CA0FDB1FA80FB91F80E09A9122914C
:1069C00030E0290F311D280F311D81E02F3F3105A7
:1069D00009F008F480E02E93615070409FEF6F3F04
:1069E000790761F7DF91CF910895EF92FF920F93AE
:1069F0001F93CF93DF938B01FC017183608361153B
:106A0000710581F022E0E22EF12CE80EF91EC0E0C3
:106A1000D0E0C7018C0F9D1F0E944D3D2196C017ED
:106A2000D107B9F7DF91CF911F910F91FF90EF90B0
:106A3000089524E030E0FC013783268384E090E071
:106A4000089521E0FC01208380E090E00895EF921A
:106A5000FF920F931F93DF93CF930F92CDB7DEB7C3
:106A60007C018E010F5F1F4FC8010E944D3D89813F
:106A70008823D1F7F7011782168280E090E00F900B
:106A8000CF91DF911F910F91FF90EF9008950F9399
:106A90001F93DF93CF930F92CDB7DEB78C01CE015A
:106AA0000196FBD78981823070F085E090E0F80193
:106AB0009783868325E030E0C9010F90CF91DF9165
:106AC0001F910F910895F8019181933141F088232E
:106AD00069F481E0F801828720E030E0EDCF88237F
:106AE00059F481E0818720E030E0E6CF86E0F801CC
:106AF000828720E030E0E0CF8DE0F801818720E060
:106B000030E0DACF0B96C9D780E090E00895CF93BC
:106B1000DF93EC016C897D898E559F4F66DF6C8910
:106B20007D89CE018B539F4F60DF80E090E0DF9145
:106B3000CF910895FC016489758981589F4F55DF75
:106B400080E090E008950F931F93CF93DF938C0123
:106B5000EC016696CE0164E070E047DFCE01C0DE56
:106B6000F801648775878687978780E090E0DF91DA
:106B7000CF911F910F9108950F931F93CF93DF93A0
:106B80008C01EC016696CE0164E070E02EDFCE0150
:106B9000A7DEF801608B718B828B938B695F7F4FCF
:106BA0008F4F9F4F28E030E040E050E00E94DE3DF4
:106BB000F801358B248B2132310564F086E090E0BA
:106BC0009783868326E030E0C901DF91CF911F9142
:106BD0000F91089520E030E0C901DF91CF911F911E
:106BE0000F910895BC0181E090E02BD780E090E008
:106BF00060E070E026D780E090E061E070E021C7BF
:106C00004F925F926F927F928F929F92AF92BF92BC
:106C1000CF92DF92EF92FF920F931F93CF93DF9368
:106C2000EC01F62E662309F4A4C08881861709F4C6
:106C3000EEC06730C1F06E30C1F48D30B1F005E0C8
:106C400010E0C801DF91CF911F910F91FF90EF905D
:106C5000DF90CF90BF90AF909F908F907F906F907C
:106C60005F904F900895863051F700E010E0A8E063
:106C7000AA2EFCE0CF2EEEE06E2E7FE0B72E62E073
:106C8000E62E992493945AE0752E45E0D42E37E0F1
:106C9000832E23E0422E99E0592EF81691F2873088
:106CA00009F495C08830A8F4833009F453C08430C7
:106CB00008F03CC08130A1F1823008F454C08F2D1F
:106CC000893008F49EC081E090E08CDF5882888192
:106CD000E4CF8B3059F08C3078F4893009F467C0F8
:106CE0008A3008F47DC09F2D9B3089F081E090E0D0
:106CF00079DFC8828881D1CF8D3009F452C08D30C0
:106D000000F18E3009F075C09F2D9B30E9F480E0D2
:106D100090E068DFF8828881C0CF8F2D813019F133
:106D200081E090E05FDFE8828881B7CF853009F4A9
:106D300044C0863090F081E090E054DF8882888102
:106D4000ACCF8F2D8D3019F381E090E04BDFB8820E
:106D50008881A3CF9F2D9430D1F281E090E042DF73
:106D6000D88288819ACF80E090E03CDF9882888149
:106D700094CF81E090E036DF00E010E080E090E02A
:106D800060E070E05ED680E090E061E070E059D6AF
:106D90000F5F1F4F0530110589F7188200E010E0E2
:106DA00050CF81E090E01EDF6882888176CF80E05E
:106DB00090E018DF7882888170CF8F2D863009F4BB
:106DC000A6CF81E090E00EDFA882888166CF9F2D5C
:106DD000943009F49CCF81E090E004DFA882F5CFE5
:106DE0008F2D813009F493CF81E090E0FBDEE882C3
:106DF0009BCF8F3009F491CFF88205E010E08881B5
:106E00004CCF80E090E0EEDE4882888146CF86302D
:106E100049F08D3009F029CF81E090E0E3DE8EE08B
:106E2000888323CF81E090E0DDDE87E088831DCF7B
:106E3000CF92DF92EF92FF920F931F93CF93DF9346
:106E4000EC018C010A5E1F4FC80161E070E0CDDDEE
:106E5000C88CC80161E070E0C8DDD88CC80164E06E
:106E600070E0C3DDC8013CDD7B018C0188858C1599
:106E700021F0CE0108966C2DC3DEC801B70123D6E0
:106E800088858D1521F0CE0108966D2DB9DE80E044
:106E900090E0DF91CF911F910F91FF90EF90DF90E5
:106EA000CF9008950F931F93DF93CF930F92CDB799
:106EB000DEB78C01CE010196F0D5C8010896698134
:106EC0009FDE9C01009719F0F80197838683C90122
:106ED0000F90CF91DF911F910F9108954F925F9284
:106EE0006F927F928F929F92AF92BF92CF92DF92DA
:106EF000EF92FF920F931F93CF93DF935B016C018F
:106F0000FA0138012115310509F481C08081918190
:106F1000D90111969C938E93808191818C010E5F93
:106F20001F4F020F131FA114B104C104D10409F4AF
:106F30005DC022E0422E512C480E591E4E0E5F1E9F
:106F40000CC00115110519F0D8019E928D01A114F4
:106F5000B104C104D10409F449C0F20182902F01A7
:106F6000EE24FF2499240894A108B108C108D1088F
:106F70006114710429F0A114B104C104D10481F198
:106F8000C82DD0E0BE016170707082E090E059D5EC
:106F900080E090E060E070E054D50115110549F003
:106FA0008ED590E00E2C02C0880F991F0A94E2F74C
:106FB000982A80E090E061E070E043D5A114B1042C
:106FC000C104D10409F4BDCF0894E11CF11CF8E020
:106FD000EF16F10409F4B5CFD595C7958C2EC3CF24
:106FE00081E090E061E070E02CD5CACFDF91CF91D5
:106FF0001F910F91FF90EF90DF90CF90BF90AF90D7
:107000009F908F907F906F905F904F9008958081B8
:10701000918100E010E087CF2F923F924F925F92D4
:107020006F927F928F929F92AF92BF92CF92DF9298
:10703000EF92FF920F931F93DF93CF93CDB7DEB7FD
:1070400028970FB6F894DEBF0FBECDBF3C01962E39
:1070500029833A834B835C831E830D8317012601AA
:10706000B886AF82A9A051E0C52ED12C681509F4CD
:1070700087C029813A814B815C8121153105410509
:10708000510529F58D8D9E8DAF8DB8A10097A10575
:10709000B10509F097C020E030E0C90128960FB68D
:1070A000F894DEBF0FBECDBFCF91DF911F910F913E
:1070B000FF90EF90DF90CF90BF90AF909F908F9018
:1070C0007F906F905F904F903F902F900895BB24DA
:1070D000EE24FF24C301692D93DD69817A818B81C0
:1070E0009C814D815E8191018601F8DE411451043D
:1070F00061F0C201B1014F8158851ADC41E0E42EF4
:10710000F12C009711F0EE24FF24C114D104E9F012
:10711000D3018C918F5F8C93E114F10459F02D8D84
:107120003E8D4F8D58A1211531054105510511F0B6
:10713000BA1448F1C301682D63DD8D8D9E8DAF8D2E
:10714000B8A10097A105B10591F4E114F10409F487
:10715000A2CFB3948B2D81508A1508F4BBCFAA20FF
:1071600019F0AB1408F439C022E030E096CFC30127
:1071700061E046DD6D8D7E8D8F8D98A1A4D4E5CF25
:10718000CC24DD2476CFC30166E03ADDC30164E0A0
:1071900037DD8D8D9E8DAF8DB8A1B595A79597954F
:1071A0008795B595A795979587952D8D3E8D4F8D94
:1071B00058A1280F391F4A1F5B1F2D8F3E8F4F8FFD
:1071C00058A3BBCFC30161E01BDD6D8D7E8D8F8D1C
:1071D00098A179D420E030E060CF23E030E05DCFAB
:1071E0008F92AF92BF92CF92DF92EF92FF920F9366
:1071F0001F93CF93DF93EC018C010A5E1F4F6C89C4
:107200007D89C801F2DB00D000D00F92288939892E
:107210004A895B89ECE5EE2EF12CEC0EFD1E79E33C
:10722000C72ED12CCC0EDD1E6FE7A62EB12CAC0ED6
:10723000BD1E8C859D85AE85BF85EDB7FEB781836C
:107240009283A383B4838B858583CE01089664E003
:107250008A84E2DE9C010F900F900F900F900F90A8
:10726000009711F09F838E83C901DF91CF911F9109
:107270000F91FF90EF90DF90CF90BF90AF908F90E5
:1072800008958F92AF92BF92CF92DF92EF92FF92CA
:107290000F931F93CF93DF93EC018C010A5E1F4F76
:1072A000C80162E070E0A1DBC8011ADB6B017C0160
:1072B000695F7F4F8F4F9F4F28E030E040E050E004
:1072C0007DD4213231058CF026E030E03F832E83DF
:1072D000C901DF91CF911F910F91FF90EF90DF9047
:1072E000CF90BF90AF908F900895C801B9017DDB1A
:1072F00000D000D00F928C859D85AE85BF85EDB7FF
:10730000FEB781839283A383B4831582CE0108964E
:107310006BE0A7019601EE24FF24CC24DD24AA24EF
:10732000BB24898479DE9C010F900F900F900F9001
:107330000F90009769F2CACF6F927F928F92AF92AF
:10734000BF92CF92DF92EF92FF920F931F93DF9342
:10735000CF930F92CDB7DEB73C01CE0101969DD3FE
:1073600083010A5E1F4F298130E040E050E0295F31
:107370003F4F4F4F5F4FF3E0559547953795279512
:10738000FA95D1F7C801B90130DB00D000D00F92D7
:10739000298130E040E050E0F30184859585A685A1
:1073A000B785EDB7FEB781839283A383B48315823B
:1073B000C30108966BE0EE24FF24CC24DD24AA242C
:1073C000BB24F301818428DE9C010F900F900F9065
:1073D0000F900F90009719F0F30197838683C901EE
:1073E0000F90CF91DF911F910F91FF90EF90DF9061
:1073F000CF90BF90AF908F907F906F9008952F9215
:107400003F924F925F926F927F928F92AF92BF9214
:10741000CF92DF92EF92FF920F931F93DF93CF9360
:1074200000D0CDB7DEB79A8389831A012B013901C9
:10743000C801B901DADAC114D10419F0C601B301E7
:10744000D4DA00D000D00F928E899F89A88DB98D93
:10745000EDB7FEB781839283A383B4838A8D85833E
:1074600089819A8164E0A2019101D6DD0F900F908D
:107470000F900F900F900F900F90CF91DF911F9171
:107480000F91FF90EF90DF90CF90BF90AF908F90D3
:107490007F906F905F904F903F902F9008958F92C4
:1074A000AF92BF92CF92DF92EF92FF920F931F9312
:1074B000CF93DF93EC0189818131D9F114E0812EE2
:1074C00000D000D00F92488959896A897B892C891C
:1074D0003D898E010A5E1F4FBCE5EB2EF12CEC0EB0
:1074E000FD1EA9E3CA2ED12CCC0EDD1EEDB7FEB7D2
:1074F00011821282138214821582CE010896AA2468
:10750000BB247DDF9C010F900F900F900F900F9088
:10751000009711F09F838E83C901DF91CF911F9156
:107520000F91FF90EF90DF90CF90BF90AF908F9032
:1075300008958A84C5CF8F92AF92BF92CF92DF9287
:10754000EF92FF920F931F93CF93DF93EC0189810A
:107550008E30A9F104E0802E00D000D00F9248892F
:1075600059896A897B892C893D898E010A5E1F4F62
:10757000EDB7FEB711821282138214821582CE01FA
:107580000896EE24FF24CC24DD24AA24BB2437DF74
:107590009C010F900F900F900F900F90009711F09B
:1075A0009F838E83C901DF91CF911F910F91FF902F
:1075B000EF90DF90CF90BF90AF908F9008958A8426
:1075C000CBCF8F92AF92BF92CF92DF92EF92FF928A
:1075D0000F931F93CF93DF93EC0100D000D00F9255
:1075E000488959896A897B892C893D898C010A5E81
:1075F0001F4FECE5EE2EF12CE80EF91E99E3C92E93
:10760000D12CCC0EDD1E8FE7A82EB12CAC0EBD1EEA
:107610008C859D85AE85BF85EDB7FEB7818392834E
:10762000A383B4838B858583CE0108968A84E7DEA5
:107630009C010F900F900F900F900F90009711F0FA
:107640009F838E83C901DF91CF911F910F91FF908E
:10765000EF90DF90CF90BF90AF908F900895CF9232
:10766000DF92EF92FF920F931F93CF93DF938C01E2
:107670006B017901B8018AD9E60128813981F701C6
:10768000A081B181AD014150504057FD38C0FD018E
:107690003296EE0DFF1D1196A00FB11F60E010E0B5
:1076A0008291882329F1EC9001E00AC0762F660FC1
:1076B0007123B1F0E02A959587958823C1F0000FDA
:1076C00090E080FFF8CF662389F721503040B60163
:1076D000620F731FEB011A8162E071E0712351F7B1
:1076E000702F7095E72295958795882341F7EC9246
:1076F0004150504011978FEF4F3F580789F6DF9167
:10770000CF911F910F91FF90EF90DF90CF90089550
:107710002F923F924F925F926F927F928F929F92A1
:10772000AF92BF92CF92DF92EF92FF920F931F938F
:10773000DF93CF93CDB7DEB761970FB6F894DEBF76
:107740000FBECDBF3C01B6E14B2E512C480E591E49
:10775000FC0164897589C20148D9C30108969D83DB
:107760008C83F301E45AFF4FFF83EE83C301C99674
:1077700099878887AFE72A2E312C260C371C00D03A
:1077800000D00F92F3012089318942895389848581
:107790009585A685B785EDB7FEB781839283A383D0
:1077A000B483F3018385EDB7FEB785838C819D811A
:1077B00064E08201EE80FF80C884D9845101F30126
:1077C00082842ADC9B838A830F900F900F900F9006
:1077D0000F90009709F087C0C3018B539F4F9D877F
:1077E0008C87FC0140815181141615060CF09DC058
:1077F000E0E0F0E060E000E010E0E60DF71DE953A6
:10780000FF4F8081882351F090E09C0121703070FF
:10781000020F131F959587958823B1F76F5FE62FA9
:10782000F0E0E417F5074CF3CE01019636D122279C
:1078300017FD2095322F095F1F4F2F4F3F4FE3E079
:107840003595279517950795EA95D1F71F870E87E8
:107850009924C30188519F4F9B878A87F301EE5576
:10786000FF4FF98BE88B8981981608F043C08A8511
:107870009B856E857F85B9D8C2016A857B854889DD
:1078800059892C853D85EBDE00D000D00F92F301A5
:10789000208931894289538984859585A685B78554
:1078A000EDB7FEB781839283A383B483F30183850D
:1078B000EDB7FEB785838C819D8164E08201EE8007
:1078C000FF80C884D9845101F3018284A5DB0F9025
:1078D0000F900F900F900F90009739F49394898137
:1078E000981640F4C4CF8A819B81F30197838683E5
:1078F0009B838A838A819B8161960FB6F894DEBF51
:107900000FBECDBFCF91DF911F910F91FF90EF90F0
:10791000DF90CF90BF90AF909F908F907F906F90AF
:107920005F904F903F902F90089500E010E07CCF43
:10793000CF93DF93EC01188219821A821B821C827A
:107940001D821F821E821B86188681E089878A8796
:10795000188A198A1A8A1B8A1D8A1C8A1C861D8607
:107960001E861F86CE01089660E04AD98E839F83CB
:10797000DF91CF910895CF93DF93EC012E813F816A
:107980002115310519F48881882321F0C901DF917F
:10799000CF910895CE01019680D08A819B81AC81E0
:1079A000BD810196A11DB11D8A839B83AC83BD83DC
:1079B000E981E83150F084E090E09F838E8324E0F9
:1079C00030E0C901DF91CF910895F0E0EE0FFF1F85
:1079D000EA5CFC4F0190F081E02DCE0109952E81EB
:1079E0003F81D4CF0F931F93DF93CF93CDB7DEB7F3
:1079F000CB50D1400FB6F894DEBF0FBECDBF8E0185
:107A00000F5F1F4FC80194DF2F8138852115310585
:107A100069F0C901C55FDE4F0FB6F894DEBF0FBE37
:107A2000CDBFCF91DF911F910F9108958981882358
:107A300081F7C801A0DF2F81388521153105B1F309
:107A4000E8CF8130910551F08230910561F00097C7
:107A500021F46115710571F442980895611571055D
:107A600039F0439A08956115710531F0459A0895EA
:107A700043980895429A08954598089580E090E0CB
:107A800060E070E0DEDF80E090E061E070E0D9CFA0
:107A900090932A38809329380895CF93DF93EC018F
:107AA000E0912938F0912A38309729F00995888398
:107AB000DF91CF9108951882DF91CF91089581E0F1
:107AC000349B80E00895AF92BF92CF92DF92EF9205
:107AD000FF920F931F935B016C0116161706180691
:107AE000190674F4EE24FF248701C8DF0894E11C12
:107AF000F11C011D111DEA14FB040C051D05ACF35E
:107B00001F910F91FF90EF90DF90CF90BF90AF90BB
:107B10000895629FD001739FF001829FE00DF11DD7
:107B2000649FE00DF11D929FF00D839FF00D749FF7
:107B3000F00D659FF00D9927729FB00DE11DF91FA3
:107B4000639FB00DE11DF91FBD01CF011124089500
:107B5000AA1BBB1B51E107C0AA1FBB1FA617B70773
:107B600010F0A61BB70B881F991F5A95A9F780958F
:107B70009095BC01CD010895A1E21A2EAA1BBB1B52
:107B8000FD010DC0AA1FBB1FEE1FFF1FA217B307E9
:107B9000E407F50720F0A21BB30BE40BF50B661FFF
:107BA000771F881F991F1A9469F7609570958095C3
:107BB00090959B01AC01BD01CF01089597FB092E63
:107BC00005260ED057FD04D0D7DF0AD0001C38F4AC
:107BD00050954095309521953F4F4F4F5F4F0895F9
:107BE000F6F790958095709561957F4F8F4F9F4FD9
:107BF00008950790F691E02D09949111089581560A
:107C00008A5108F4805285580895FB01DC010590E3
:107C10000D920020E1F70895FC0105900020E9F79E
:107C2000809590958E0F9F1F0895FB01DC0104C085
:107C30008D910190801921F441505040C8F7881B64
:107C4000990B0895FB01DC0102C001900D92415097
:107C50005040D8F70895FB01DC014150504030F00E
:107C60008D910190801919F40020B9F7881B990BA8
:107C70000895FB01DC014150504048F001900D9205
:107C80000020C9F701C01D9241505040E0F708950F
:107C90000F931F93DF93CF93CDB7DEB72E970FB619
:107CA000F894DEBF0FBECDBF0D891E898F89988DD8
:107CB00026E02C831A83098397FF02C080E090E8B6
:107CC00001979E838D839E01255E3F4FCE010196D5
:107CD000698D7A8DA90119D04D815E8157FD0AC049
:107CE0002F813885421753070CF49A01020F131F96
:107CF000F80110822E960FB6F894DEBF0FBECDBFEE
:107D0000CF91DF911F910F9108952F923F924F9243
:107D10005F926F927F928F929F92AF92BF92CF921B
:107D2000DF92EF92FF920F931F93DF93CF93CDB724
:107D3000DEB72C970FB6F894DEBF0FBECDBF6C0137
:107D40001B018A01FC0117821682838181FFC4C155
:107D50002E010894411C511CF6019381F10193FD01
:107D6000859193FF81911F01882309F4B1C1853268
:107D700039F493FD859193FF81911F01853221F4A0
:107D800090E0B601F5D1E8CFEE24FF2420E02032C8
:107D9000B0F48B3269F08C3228F4803251F08332A7
:107DA00071F40BC08D3239F0803349F421602CC05E
:107DB0002260246029C0286027C0206125C027FDDB
:107DC0002CC0382F30533A3098F426FF08C08E2D3F
:107DD000880FE82EEE0CEE0CE80EE30E15C08F2D8A
:107DE000880FF82EFF0CFF0CF80EF30E20620CC06B
:107DF0008E3221F426FD6CC1206406C08C3611F44D
:107E0000206802C0883649F4F10193FD859193FF03
:107E100081911F01882309F0BACF982F9554933090
:107E200018F09052933028F40C5F1F4FFFE3F98352
:107E30000DC0833631F0833771F0833509F05CC0B3
:107E400021C0F801808189830E5F1F4F420171E0DC
:107E5000A72EB12C15C062E0662E712C600E711E2B
:107E6000F8018080918026FF03C06E2D70E002C073
:107E70006FEF7FEFC4012C8770D15C0183012C85EB
:107E80002F7716C052E0652E712C600E711EF8011E
:107E90008080918026FF03C06E2D70E002C06FEFDE
:107EA0007FEFC4012C874ED15C012C8520688301B3
:107EB00023FD1EC007C080E290E0B6012C8758D198
:107EC000FA942C858F2D90E0A816B906A0F310C067
:107ED000F40127FD859127FF81914F0190E0B601C4
:107EE0002C8746D12C85F110FA940894A108B1088A
:107EF000A114B10469F7E9C0843611F0893641F55F
:107F000027FF08C0F80160817181828193810C5F35
:107F10001F4F09C0F80160817181882777FD809526
:107F2000982F0E5F1F4F4FE6B42EB22297FF09C065
:107F300090958095709561957F4F8F4F9F4FF0E89A
:107F4000BF2AA2012AE030E03FD1782E741844C045
:107F5000853731F43FEEB32EB2222AE030E025C05F
:107F600099EFB92EB2228F36C1F0803720F48835D0
:107F700009F0AEC00DC0803721F0883709F0A8C0E5
:107F800002C020E1B22AB4FE0BC084E0B82A08C0C7
:107F9000B4FE09C0E6E0BE2A06C028E030E005C015
:107FA00020E130E002C020E132E0B7FE08C0F80175
:107FB00060817181828193810C5F1F4F07C0F8013E
:107FC0006081718180E090E00E5F1F4FA201FCD0C4
:107FD000782E7418FFE7BF22B6FE0BC02EEFB22238
:107FE0007E1438F4B4FE07C0B2FC05C08FEEB82290
:107FF00002C0A72C01C0AE2C8B2D90E0B4FE0DC0AA
:10800000FE01E70DF11D2081203319F4E9EEBE22B7
:1080100009C0A394B2FE06C004C086789070009791
:1080200009F0A3948B2C9924B3FC13C0B0FE0EC0AE
:10803000AF1428F4E72CEF0CEA18AF2C07C0E72C9C
:1080400005C080E290E0B60193D0A394AF14C8F3CA
:1080500004C0AF1410F4FA1801C0FF2484FE0EC04F
:1080600080E390E0B60184D082FE1DC081FE03C093
:1080700088E590E010C088E790E00DC0C4018678E4
:108080009070009781F081FC02C080E201C08BE219
:10809000B7FC8DE290E0B6016BD005C080E390E0C4
:1080A000B60166D0EA947E14C8F37A94F201E70D23
:1080B000F11D808190E0B6015BD07720B1F705C05B
:1080C00080E290E0B60154D0FA94FF20C9F744CE84
:1080D000F6012681378102C02FEF3FEFC9012C96B0
:1080E0000FB6F894DEBF0FBECDBFCF91DF911F91C9
:1080F0000F91FF90EF90DF90CF90BF90AF909F9047
:108100008F907F906F905F904F903F902F90089549
:10811000F999FECF92BD81BDF89A992780B508954F
:10812000262FF999FECF92BD81BDF89A019700B430
:10813000021639F01FBA20BD0FB6F894FA9AF99AD0
:108140000FBE0895FC010590615070400110D8F7F2
:10815000809590958E0F9F1F0895FC01615070408F
:1081600001900110D8F7809590958E0F9F1F08956C
:108170000F931F93CF93DF938C01EB018B8181FFD2
:108180001BC082FF0DC02E813F818C819D812817ED
:10819000390764F4E881F9810193F983E88306C023
:1081A000E885F985802F0995009731F48E819F81AC
:1081B00001969F838E8302C00FEF1FEFC801DF91EE
:1081C000CF911F910F910895FA01AA27283051F1FC
:1081D000203181F1E8946F936E7F6E5F7F4F8F4FF8
:1081E0009F4FAF4FB1E03ED0B4E03CD0670F781F57
:1081F000891F9A1FA11D680F791F8A1F911DA11D3C
:108200006A0F711D811D911DA11D20D009F4689474
:108210003F912AE0269F11243019305D3193DEF61C
:10822000CF010895462F4770405D4193B3E00FD0D2
:10823000C9F7F6CF462F4F70405D4A3318F0495DBD
:1082400031FD4052419302D0A9F7EACFB4E0A695A0
:108250009795879577956795BA95C9F700976105C2
:10826000710508959B01AC010A2E06945795479518
:1082700037952795BA95C9F7620F731F841F951F0D
:10828000A01D089518E000E0C8E9D8E040E005C06E
:1082900022974109FE014BBFACDCCA39D107400728
:0682A000B9F7F894FFCFCE
:1082A6002E2E0053656C656374204469736B006EF3
:1082B6006F20696D6167652066696C657320666FFE
:1082C600756E640001030507090E10121416181CBA
:1082D6001E696E636F6D706C657465207772697464
:1082E600650062616420736563746F722025642083
:1082F600666F722074256400627566206C6F636B0E
:1083060065642025642F25643A25640063686563E7
:108316006B73756D206661696C75726520300063DC
:108326006865636B73756D206661696C757265202F
:108336003100636865636B73756D206661696C7582
:108346007265203200636865636B73756D206661C4
:10835600696C006669726D776172652E7876660063
:10836600524553554C543A205355434345535300B5
:108376004649524D57415245204552524F522025AB
:10838600640043504C44204669726D7761726520E3
:1083960025640025640025750053442072656164D8
:1083A600206572726F722052004241442046555336
:1083B600455320253032582025303258202530327A
:1083C600580043504C4420495320424C414E4B00E8
:1083D60057524F4E472043504C44202D20256400D1
:1083E60053454C462D54455354204F4B005344207F
:1083F60072656164207374617274206572726F7243
:108406000053442072656164206572726F72204465
:108416000077722077726F6E6720747261636B20CB
:1084260025642F2564005265766572746564207430
:10843600726B202530326420202000534420726560
:108446006164206572726F72205700534420777200
:108456006974655374617274206661696C00534473
:10846600207772697465206572726F7200534420BA
:10847600777269746553746F70206661696C005316
:10848600617665642074726B202530326420696ED3
:1084960020256C752020004E4F2053442043415226
:1084A600443F0043415244204552524F52202564D6
:1084B6003A256400253032640025642000D5AAAD33
:1084C6000000000000000000000000008A01AD016D
:1084D600D8010D024E0221359A359C39F038A33564
:1084E600193519358235BC35E13A8735883B9B3AD3
:1084F6009B3A9B3A4F3A4F3A4F3A523747354735B0
:068506004139273518374A
:020000021000EC
:08EFF800DDDDDDDD000100009C
:00000001FF
